:100000000C9466000C9487000C9487000C94870075
:100010000C9487000C9487000C9487000C94870044
:100020000C9487000C9487000C9487000C94870034
:100030000C9487000C9487000C9487000C94870024
:100040000C9487000C9487000C9487000C94870014
:100050000C9487000C943F0D0C9487000C9487003F
:100060000C9487000C94D6110C9487000C94870094
:100070000C9487000C9487000C9487000C948700E4
:100080000C9487000C9487000C9487000C94060E47
:100090000C94AA190C9487000C9487000C94870088
:1000A0000C9487000C9487000C9487000C948700B4
:1000B0000C9487000C9487000C9487000C948700A4
:1000C0000C9487000C9487000C94870011241FBEA9
:1000D000CFEFD1E2DEBFCDBF00E00CBF14E0A0E067
:1000E000B2E0ECE5FCE800E00BBF02C007900D9227
:1000F000AE32B107D9F717E0AEE2B4E001C01D920D
:10010000A631B107E1F70E94B9030C942C460C9478
:100110000000109234048091340480933304809161
:10012000330480933204809132048093310410921E
:1001300035040895EEE6F0E080818260808383E0FC
:1001400084BD85BD8AEF87BD0895E1E7F0E0808139
:1001500081608083089580917100817008958091FD
:100160008904982F9295969596959370282F221F23
:100170002227221F9227282F22952F709227282F7F
:100180002695269592279170880F892B8093890454
:10019000089590937F0480937E0485EB9BE3909376
:1001A00091048093900483E393E190939704809368
:1001B000960485E694ED90938D0480938C040895C5
:1001C00080917E0490917F04AC01440F452F441F21
:1001D000550B5195482759276091900470919104CF
:1001E00070937F0460937E048091960490919704AD
:1001F000909391048093900420918C0430918D040D
:100200003093970420939604C9010024969587950E
:100210000794969587950794982F802D822793278A
:1002200084279527542F44275295550F507E8427B5
:10023000952790938D0480938C04660F771F6F5FD2
:100240007F4F869F9001879F300D969F300D112420
:10025000C9010895FC019081992351F08091C80053
:1002600085FFFCCF9093CE00319690819923B1F712
:1002700008951F93CF93DF93182F492FE0E1F7E202
:10028000C0E0D0E0812F942FBF010E94E3459B0185
:100290006115710589F5812F942FBF010E94E345F7
:1002A000182F492FCF016AE070E00E94E345FB015F
:1002B0002196C430D10531F73097A1F18091C80063
:1002C00085FFFCCF812F942FBF010E94E345605D25
:1002D0006093CE00CF016AE070E00E94E3459B018D
:1002E00061157105F9F0812F942FBF010E94E3453C
:1002F000182F492FF901E2CF8091C80085FFFCCF6C
:10030000822F805D8093CE00812F942FBF010E94A9
:10031000E345182F492FCF016AE070E00E94E345C2
:10032000FB01CACFDF91CF911F910895982F9F7045
:100330009A3040F48091C80085FFFCCF905D909387
:10034000CE0008958091C80085FFFCCF995C909302
:10035000CE000895CF93DF93EC01892F99278295E2
:100360008F700097C1F48D2F9927009789F4CE01E3
:10037000929582958F7089279F708927009711F039
:100380000E9496018C2F0E949601DF91CF910895D3
:100390000E949601ECCF0E949601E5CF982F8091A4
:1003A000C80085FFFCCF9093CE0080E090E00895D8
:1003B0002091C800332727FD30952227330F221FB5
:1003C0003327C90108958091C80087FFFCCF809131
:1003D000CE0090E008959C018FEF8093830493E01A
:1003E000283E390768F58093800480938104243681
:1003F0003105D8F0C90164E670E00E94E3456093DE
:100400008004C9016AE070E00E94E345CB016AE024
:1004100070E00E94E34580938104C9016AE070E0C6
:100420000E94E3458093820408952A30310548F7FD
:10043000C9016AE070E00E94E34580938204089558
:100440001092800410928104109282040895909179
:100450003604936090933604809337040895809116
:1004600036048360809336040895F999FECF92BDD7
:1004700081BDF89A30B5F999FECF019692BD81BD44
:10048000F89A20B5932F80E030E0282B392BC90152
:100490000895F999FECF92BD81BDF89A80B508956F
:1004A000F999FECF92BD81BD60BDF894FA9AF99A90
:1004B00078940895FF920F931F938C01F62E672F67
:1004C0000E945002C80101966F2D0E9450021F9198
:1004D0000F91FF9008958091C90088618093C900B1
:1004E00083E38093CC001092CD008091C80087FDFB
:1004F00032C08091C90080688093C9008091C1009A
:1005000088698093C1008FE18093C4001092C50078
:1005100090EC91B98CE382B987E384B995B99FEFE8
:1005200097B988EF8AB98BE08BB982E08DB99EB913
:1005300010BA91BB13BA94BB8DB581608DBD81E5B6
:100540008CBD08958091CE008AE00E94420E809179
:10055000C80087FFCECF8091C80087FDF3CF809180
:10056000C80087FFF8CFEECFEF92FF920F931F9353
:10057000CF93DF93EC0181E0CD32D80750F5C8323C
:10058000D105B0F588E290E090937B0480937A04E3
:1005900090938804809387040E94651924E234EFC5
:1005A00030938B0420938A0482E0809391008091A1
:1005B0008A0490918B04909581959F4F90938B0422
:1005C00080938A04DF91CF911F910F91FF90EF905C
:1005D00008958CE291E090937B0480937A04909349
:1005E0008804809387040E9465192DE830E2D8CFF3
:1005F000D0937B04C0937A04D0938804C09387047B
:10060000CE010E9465199E0140E050E060E070E775
:1006100088E399E30E940A46B901CA019695879535
:10062000779567959695879577956795969587952C
:100630007795679526E030E040E050E00E940A465A
:1006400079018A01C801AA27BB279C01887F892BD1
:1006500009F45FC0C901807F892B99F0C901807EB0
:10066000892BF1F0C901807C892B49F1C901807087
:10067000892BA1F120703C7F232BE1F11092910096
:1006800096CFF4E016950795F794E794FA95D1F78D
:10069000F0928B04E0928A0486E08093910087CFE9
:1006A000E5E016950795F794E794EA95D1F7F0926F
:1006B0008B04E0928A0487E08093910078CF76E003
:1006C00016950795F794E7947A95D1F7F0928B04F5
:1006D000E0928A0483E08093910069CFBB27A12F29
:1006E000902F8F2D90938B0480938A0484E08093C5
:1006F00091005DCF5AE016950795F794E7945A95C7
:10070000D1F7F0928B04E0928A0485E08093910007
:100710004ECFA3E016950795F794E794AA95D1F7E5
:1007200097013ECF85E090E00E9435020E94B4021E
:1007300080918A0490918B0490937D0480937C0433
:1007400010922F04E1E7F0E0808181608083809146
:100750007A0490917B0490938F0480938E04089583
:1007600085E20E948B15E1E7F0E080818E7F808337
:100770000895AF92BF92CF92DF92EF92FF920F93C4
:100780001F93DF93CF93CDB7DEB760970FB6F89482
:10079000DEBF0FBECDBF0E946B020E94920380910C
:1007A0006E00826080936E0083E084BD85BD8AEF19
:1007B00087BD89E696E09093AC068093AB06F999E5
:1007C000FECF82E090E092BD81BDF89A80B5982F6F
:1007D000937090932E048295817080936804F999A8
:1007E000FECF87E090E092BD81BDF89A80B5882366
:1007F00011F0813208F080E180930002F999FECF78
:1008000083E090E092BD81BDF89A80B58F708093AF
:10081000AB04F999FECF84E090E092BD81BDF89AD7
:1008200080B58F708093980488E090E00E94350234
:100830008093890420917A0430917B04280F391F1A
:1008400030937F0420937E0485EB9BE39093910487
:100850008093900483E393E19093970480939604AC
:1008600085E694ED90938D0480938C040E94E000C3
:100870000E94E0000E94E000BC0188E090E00E943D
:100880005A02F999FECF8AE090E092BD81BDF89AB4
:1008900090B5892F8F708093920480919204833059
:1008A00010F01092920492959F709F5F9093950420
:1008B00080919504823008F4E2C00E94E12C789483
:1008C00000E010E01DC08091D8040E9425160E940F
:1008D0005717C801849668E270E00E94F7450E94AD
:1008E000ED180E948B1580E10E94420EC8018770AE
:1008F0009070892B69F00F5F1F4F0C32110579F052
:10090000083208F7802F0E94ED180E945315DBCFA4
:100910000E94A6140F5F1F4F0C32110589F70E9429
:1009200002160E9457170E94A61480E00E94E1124E
:10093000882331F083E00E94E112882309F0EBC0A4
:1009400083E00E94E112882309F09DC08091D804C1
:100950008093C206109203071092960510921F060C
:1009600081E080932506109226068091C206609150
:10097000030740911F062091250609E616E00E9414
:10098000E72B60911F06C8010E9420290E94AB2816
:100990000E94A614809136048360809336041092DE
:1009A00037048091D304873009F466C0883030F56D
:1009B000823009F449C08330A8F5882309F44AC07D
:1009C000813009F444C00E94A6140E94AB288823F9
:1009D000F9F68091D3048630B1F781E00E940D13BF
:1009E000882389F380E00E94E112882361F30E944A
:1009F00002160E945717E0E0F0EF19948C30C9F10D
:100A00008D3038F4883061F18B30E9F60E9438225D
:100A1000BFCF8E3011F18E30A0F08F30A1F60E9442
:100A2000F72CB6CF843051F0843028F0853059F659
:100A30000E940B32ADCF0E94C924AACF0E94DE1CB7
:100A4000A7CF0E94A044A4CF0E94203CA1CF0E9427
:100A50003B3E9ECF0E946F119BCF0E94401998CFC2
:100A60000E9402160E94A6140E94AB288823D1F38C
:100A70008FCF0E94ED0F8CCF0E94802689CF82E01D
:100A8000809395041ACF8CE00E94E112882309F428
:100A90005DCF7E010894E11CF11CBB2491E1C92EBD
:100AA000D12CCC0EDD1E8FE0A82E87010E94E00025
:100AB000F801908381830E5F1F4F0C151D05B1F760
:100AC000F70104C031960E171F0791F02081822F85
:100AD00090E08F7090700D9724F0822F8F7080833C
:100AE000282F2D3079F78E2F8E198F3009F072C094
:100AF00080E060E04B2D21E087010E945C2C85E5C1
:100B00000E940C190E945717B394F0E8BF1669F6BB
:100B10000E9402161BCF10922E041092680460915E
:100B2000680470E06170707062957295707F7627CE
:100B3000607F762782E090E00E9450020E94E12CC4
:100B40001092AB041092980483E090E060E00E9461
:100B5000500284E090E0609198040E94500288E77F
:100B600090E090937B0480937A0485E090E068E7BE
:100B700070E00E945A0280E18093000260910002BE
:100B800087E090E00E9450021092920488E08093E7
:100B90009504809195046091920490E0019782956C
:100BA0009295907F9827807F9827682B8AE090E025
:100BB0000E94500210E082E20E94BF1583E20E9470
:100BC000BF150E94571782E30E94420E1F5F183222
:100BD00091F79ECFA08276CFCF92DF92EF92FF92D5
:100BE0000F931F93CF93DF93F89480912E0481305D
:100BF00009F4DEC280917104813009F40BC2809146
:100C00003104863060F010923104809132048F5F9D
:100C100080933204809133048F5F809333048091FA
:100C20003304882341F08091330490E08370907006
:100C3000892B09F4D8C180913404883038F010929F
:100C4000340480912E04882309F4ACC180913304CC
:100C50008F70809333049091320480910002981732
:100C6000C0F010923204809135048F5F8093350478
:100C70009091350480919504981708F090C1809167
:100C8000360482608093360480913A0481608093B8
:100C90003A0480911007882329F480913204882334
:100CA00009F473C180913204882329F4809171047E
:100CB000823009F45CC28091D3048C3009F499C16C
:100CC00080912E04882301F5909143048091E903DB
:100CD000981710F0109243048091430480FF58C28B
:100CE0005C988091430480FF0FC0809143048F5F24
:100CF000809343047894DF91CF911F910F91FF90DF
:100D0000EF90DF90CF900895809172042091E903D5
:100D10004091E90390E030E0240F311D82179307E2
:100D200014F010927204809172046091E903669548
:100D30000E94D745992309F48CC0DD248091D30407
:100D4000873009F492C0883008F082C1813008F001
:100D500024C280917104823009F454C2809110073A
:100D6000882321F082E0D81609F457C28091100739
:100D7000882309F419C280915E048F7080935E0409
:100D80008091330490E08370907002970CF4CEC190
:100D900085E20E948B1580915E0490E083709070D4
:100DA00002970CF4C0C18FEF8093560480916704C2
:100DB000882309F088C180917004882329F08091EC
:100DC0003704882309F0B6C180913804882309F0DC
:100DD00068C10E945717DD2031F080912F048F5F8A
:100DE000817080932F042091870430918804809132
:100DF0007A0490917B042817390729F080912E04FA
:100E0000882309F4FBC1809172048F5F8093720480
:100E1000809104078F5F80930407809131048F5F76
:100E200080933104809143048F5F80934304209129
:100E300004078091E90330E0869586954CE0849F15
:100E4000C00111242817390714F010920407789470
:100E500052CF80912F04882309F486C1DD24D394D6
:100E60008091D304873009F06ECF81E0D81609F461
:100E7000B6C2E2E0DE1609F06CCF80915E048F5FAF
:100E800080935E0480911007882309F478C08091D4
:100E90009705882309F51092040780919B05882304
:100EA00049F480910607882329F0809167048823FC
:100EB00009F094C580911F0660916706680F8091C4
:100EC000AB069091AC060E94202910925E0480919E
:100ED0006204882309F4CBC480919705E091AB06A6
:100EE000F091AC06E80FF11D808180937904809128
:100EF00086048093840480917904807480938604AE
:100F000080916704882309F046C4809179048F702A
:100F10008F3009F4A2C4809179048F708F3029F149
:100F2000809179040E9444290091B106080F109124
:100F30007904107860918404802F412F0E94BF1C97
:100F4000112309F092C480E0902F935F982B809139
:100F50003B04981751F080913B0480933C0490939C
:100F60003B0480913B040E94010F8091D3048330A5
:100F700009F420C48091D304873009F4E6C380913A
:100F80003604816080933604E4CE8091710482300F
:100F900009F088CE109271040E94243083CE109202
:100FA00035046DCE20917A0430917B0480918E04BB
:100FB00090918F042817390709F448CE80911007C3
:100FC000882309F043CE85E20E94531560917A048C
:100FD00070917B0470938F0460938E0485E090E0A1
:100FE0000E945A0233CE809134048F5F8093340480
:100FF00022CE80913A0480FF0AC080911007882396
:1010000009F093C180913F04882309F019C310921D
:101010003A0456CE80911007882309F0B6C00E948A
:10102000243080912E04882381F41092340480911E
:10103000340480933304809133048093320480918C
:101040003204809331041092350410927104D7CD8C
:101050008B3009F40ACF8C3008F0E3C0883009F0F7
:1010600078CEF1E0DF1609F446C382E0D81609F025
:1010700070CE8091780480933004809177048093BF
:1010800078040E94AF0080937704809178048F7376
:1010900060E040E00E94BF1C809178040E94010F34
:1010A00058CE0E94FE188091330480FD92CEE091CC
:1010B0003304E695F0E0E370F070E058FB4F808178
:1010C0000E94F31886CE8CE20E944429982F8091CA
:1010D0005E048111945F80910407882341F480911C
:1010E0006804882309F401C383E20E9453158091A8
:1010F0000407823009F05FCE80916804882379F478
:1011000080916504823008F40BC3809123060E940D
:10111000442940912306407860E00E94BF1C83E28E
:101120000E948B1548CE1092560440CE85E20E9454
:10113000531531CE80919204813009F440C18091E1
:101140009204882309F040CE8091360480FF3CCE83
:10115000809136048E7F809336040E94171680910A
:1011600097050E94251630CEB2E0DB2EE7CD8091A8
:10117000D304853009F49FCD1092720410922F048D
:10118000109297051092710496CD0E94E32F5DCFC7
:101190005C9A88EF0E944D0FA4CD843008F465CE90
:1011A000853009F0D6CD61CE81E20E948B15E3CD6A
:1011B0000E9468128823A9F080917004882309F0A6
:1011C000A4C210923404809134048093330480913B
:1011D000330480933204809132048093310410925E
:1011E00035040E947A12882309F404CD809170049A
:1011F000882309F4FFCC0E94E32FFCCCC9010E9494
:10120000B40201CE81E20E948B158091310463E02B
:101210000E94D745992309F0AECD81E20E94531573
:10122000AACD8C3021F08D3009F093CD1ECE0E94D6
:10123000171680913A0480FDFFC180913F048823F6
:1012400009F0F4C1E1E0DE1609F483C1F2E0DF1633
:1012500009F07FCD80915E048F5F80935E04809162
:101260001007882309F475CDE0916706F0E0E35597
:10127000F94F808184FD5FC286E08093E90380910D
:101280009705E091AB06F091AC06E80FF11D808167
:1012900080937904809186048093840480917904FA
:1012A000807480938604809179048F708F3009F464
:1012B0006AC2809179048F708F3071F080917904C7
:1012C0000E9444299091B106609184044091790470
:1012D0004078890F0E94BF1C80913904982F929505
:1012E0009F709093C206982F977090931F068695D3
:1012F00086958695817080930307809103078823E4
:1013000009F012C288E00E94531581E00E948B15FB
:101310000E94001780911F068F5F0E94A016809187
:10132000100781708093100714CD809110078230D0
:1013300008F46DCE80913F04882329F480918305C1
:10134000882309F464CE80914004809339049091FD
:1013500067069F5F909367069091670691709093E0
:1013600067066091670670E062957295707F7627D8
:10137000607F76276759794F7093AC066093AB0610
:1013800090916706C92FD0E00E948A2BC355D94F90
:101390008883E0916706F0E0E355F94F80818F7014
:1013A0008F5F8093EB03E0916706F0E0E355F94F20
:1013B000808184FDA8C186E08093E90328CE8091D6
:1013C000360481FFBCCE809136048D7F8093360435
:1013D0000E941716809135040E942516B0CE809188
:1013E0009B058F5F80939B0580911007882309F4EC
:1013F000B0CC809197058F5F80939705909197056A
:101400008091EB03981710F0109297058091970543
:10141000882309F06EC08091D304833009F44AC157
:1014200010E08091D304873009F4D1C181E00E949B
:10143000EF28809167068F5F80936706C0906706EC
:101440009091670680912506981708F443C0809113
:101450006204882319F481E080936F048091D3049F
:10146000813009F41BC28091D304823009F412C286
:1014700082E00E94EF2810929B05809167048823E8
:1014800069F08091650480930607809106078823A0
:1014900029F01092650481E080939505109267060B
:1014A0008091D304833009F436C28091D30487300D
:1014B00009F40BC280912606882309F0F2C19091AD
:1014C000030780919605981729F080916204823075
:1014D00008F4B8C28091670690E082959295907F5B
:1014E0009827807F98278759994F9093AC068093CF
:1014F000AB0680916704882309F02BCC8091970577
:10150000E091AB06F091AC06E80FF11D808180936D
:101510007904809179048F708F3009F49BC1809198
:1015200086040E94D61C80913C04882309F08BC15C
:1015300080918604882309F00CCC80913B04882399
:1015400009F407CC80913B040E94270F10923B04C2
:1015500000CC80911007882309F4FBCB809197057C
:101560008F5F8093970580913F04882309F4D0C052
:1015700090914004809139048917D1F1F090670669
:10158000F394FE220F2D10E0E801C295D295D07F92
:10159000DC27C07FDC27C759D94F80914004BE01AA
:1015A0000E948A2B0355194FF8018083E09167064A
:1015B000F0E0E355F94F2081F801808190E030E0C0
:1015C0008227932784FD14C08091400480933904BE
:1015D000F0926706E0916706F0E0E355F94F8081ED
:1015E0008F708F5F8093EB03D093AC06C093AB06F4
:1015F000809197056091EB030E94D74590939705E2
:1016000080919705E091AB06F091AC06E80FF11DD3
:10161000808180937904809179048F708F3009F4F0
:101620008CC0809186040E94D61C93CB80913F048D
:1016300081500E94251606CE8FE00E942516FDCD12
:1016400080914004809339040E94243080912E04BC
:10165000882381F4109234048091340480933304FD
:10166000809133048093320480913204809331045A
:1016700010923504809167068F5F80936706809192
:1016800067068170809367066091670670E06295D7
:101690007295707F7627607F76276759794F7093B0
:1016A000AC066093AB0680916706C82FD0E08091AE
:1016B00039046ACE80917F059091800501969093C0
:1016C000800580937F0520917F0530918005809172
:1016D0008A0590918B052817390708F4A1CE10923E
:1016E000800510927F0511E09CCE892F60E040E0DC
:1016F0000E94BF1CF9CC80E00E94D61C8091780427
:101700000E94270F26CB88E057CE0E94243059CD67
:1017100080918305882309F06BCF0E94E32F68CF67
:1017200080E00E94D61CFBCC88E00E948B1581E0F3
:101730000E945315EDCD88E0A0CD809186048823CA
:1017400009F0A4C0109286046CCF809138048130D7
:1017500009F43CC180917F0590918005E09190054E
:10176000F0E0EE0FFF1FEF5FFD4F6081718182950A
:101770009295907F9827807F98270E94E345862F37
:101780000E943016FCCB809179048F70809379048D
:10179000109286048ECD80911F066091250640919F
:1017A00098052091260600919C05E09096050E94E0
:1017B0004618DBCB80913804813009F0DBCB809177
:1017C0007F059091800501960E94EB01D3CB80911B
:1017D0005D04813009F02ACE6091030780911F06D5
:1017E000409167062091B106480F87E895E00E9476
:1017F0003C1E8091900560917F057091800540911D
:1018000087050E94A21E80917F0590918005019618
:101810009093800580937F05E091900520917F054E
:1018200030918005F0E0EE0FFF1FEF5FFD4F8081EC
:1018300091812817390708F4F9CD10925D0483E2ED
:101840000E948B15F3CD80913C040E94270F1092CB
:101850003C046ECE1092860462CE809179048F7023
:10186000809379041092860456CB80E86DCB8091EA
:101870001F0660912506409198052091260600914B
:101880009C05E09096050E94461826CB81E00E94B8
:10189000D61C58CF81E080936F04EACD80936F040B
:1018A000E2CD0E94DC2880916204823008F012CEE2
:1018B0008091C2066091030740911F062091250682
:1018C00009E616E00E94E72B05CE80915D04813089
:1018D00009F0F0CD80918305882309F0B8C080918C
:1018E0008405882309F4E6CD109284058091900543
:1018F00060917F05709180056C190E94691E80912E
:1019000090050E94FC1E909392058093910580E0C3
:101910000E948B15CFCD80918305882309F079C073
:1019200080918405882309F44EC01092800510929E
:101930007F058091CE0480939005809190050E9450
:10194000051F90938B0580938A05809190050E94D6
:10195000FC1E909392058093910520919105309102
:10196000920580918A0590918B052817390720F000
:10197000109292051092910580918405882309F0B8
:1019800053C08091900560917F05709180050E9401
:10199000561F8093870580919005609187054EEDD5
:1019A00055E026E935E008E915E0EAEAEE2EE6E042
:1019B000FE2E0E941C1E81E0809326068091AA06BE
:1019C0008093B10672CD1123B9F2AFCF80917F051C
:1019D0009091800501960E94EB01BCCE81E00E94AF
:1019E000D61C80E00E94D61C6091250689E696E010
:1019F00043EC56E02DE935E00E944F2A109267042F
:101A00008AE00E9460291092860482E00E94420EC1
:101A100051CA109283051092800510927F0583E2CF
:101A20000E948B1511E07CCF109284058091910566
:101A3000909192059093800580937F0580E00E94AD
:101A40008B159FCF809196058093030731CF10921D
:101A50005D04109283058091900560917F057091DF
:101A600080050E94791E809190050E94051F909329
:101A70008B0580938A0583E20E948B1530CF1F92DD
:101A80000F920FB60F920BB60F9211242F933F9324
:101A90004F935F936F937F938F939F93AF93BF9376
:101AA000EF93FF9320B1227090B180919404281796
:101AB000F1F0892F8170222309F479C0882309F479
:101AC00079C080918704909188040197909388044D
:101AD0008093870431E08D32930708F479C08CE25B
:101AE00091E09093880480938704209394048091DC
:101AF0004A048F3F29F080914A048F5F80934A0403
:101B000080914B048F3F29F080914B048F5F80932D
:101B10004B0480917504909176048F5F9F4F49F03C
:101B20008091750490917604019690937604809349
:101B300075048091590490915A048F5F9F4F49F02A
:101B40008091590490915A04019690935A0480937D
:101B5000590420912E04213009F444C0809144049A
:101B600090914504892B81F0809144049091450423
:101B7000019790934504809344048091440490918C
:101B80004504892B09F45C98FF91EF91BF91AF91C7
:101B90009F918F917F916F915F914F913F912F9185
:101BA0000F900BBE0F900FBE0F901F9018958823BB
:101BB00009F487CF809187049091880401969093CF
:101BC00088048093870431E08D32930708F087CF33
:101BD000889708F08ACF88E290E0909388048093F9
:101BE000870483CF99B1929591708091480488239E
:101BF00019F090934804C8CF9923D9F3209348044F
:101C00000E94EC0588EF0E944D0FBECF1F920F92ED
:101C10000FB60F920BB60F9211242F933F934F9351
:101C20005F936F937F938F939F93AF93BF93EF9344
:101C3000FF9380917C0490917D0490939500809314
:101C4000940080918A0490918B0490937D048093FA
:101C50007C0480912E04882311F40E94EC05FF91EE
:101C6000EF91BF91AF919F918F917F916F915F9114
:101C70004F913F912F910F900BBE0F900FBE0F9081
:101C80001F90189520EA3FE0E22FF32F3197F1F7EC
:101C90008A95D1F70895882309F41EC09AEF20EAA7
:101CA0003FE0E22FF32F3197F1F79A95D1F7E22F2A
:101CB000F32F3197F1F79A95D1F7E22FF32F319760
:101CC000F1F79A95D1F7E22FF32F3197F1F79A9523
:101CD000D1F7815009F0E5CF08951092A104109238
:101CE000AA0408951F93CF93DF93EC01142F6F770D
:101CF0007885772309F44CC0462F50E0888190E026
:101D00008F7790704817590779F121E030E00DC0C6
:101D1000D901FE01E20FF31F808190E08F77907070
:101D20002F5F3F4F8417950709F1271788F3272F57
:101D30002F5F293030F128E0922F822F9150FE0141
:101D4000E80FF11DDE01A90FB11D8C918083892F51
:101D50009923A1F71536C0F480E0862B8883288765
:101D6000DF91CF911F910895A0E0B0E0153670F497
:101D700080E0AC0FBD1F862B8C93DF91CF911F911C
:101D800008952223C9F6E6CF80E8E7CF80E8F1CFB7
:101D900091E081E021E0D2CFCF93DF93EC01388551
:101DA0003323B9F06F7770E0888190E08F7790707F
:101DB0006817790789F0FE0120E008C0818190E072
:101DC0008F77907031966817790739F02F5F231756
:101DD000A8F3DF91CF91089520E0323068F0922F80
:101DE0009F5FFE01E20FF11DDE01A90FB11D8C9175
:101DF0008083292F9317A0F331503887DF91CF913B
:101E00000895282F909198048091C00085FFFCCF01
:101E100090699093C6008091C00085FFFCCF822F0F
:101E20008F778093C60027FD09C09091230280918F
:101E3000C00085FFFCCF9093C600089590912102C9
:101E40008091C00085FFFCCF9093C6000895282F95
:101E5000909198048091C00085FFFCCF906890938A
:101E6000C6008091C00085FFFCCF822F8F778093C2
:101E7000C60027FD09C0909123028091C00085FF14
:101E8000FCCF9093C6000895909121028091C000EC
:101E900085FFFCCF9093C6000895982F8091C000D5
:101EA00085FFFCCF9093C60080E090E0089590916C
:101EB00041048091420420E030E0981711F021E0C5
:101EC00030E0C9010895909141048091420498172F
:101ED000D1F3F89490914104E92FF0E0E455FB4FE1
:101EE00080819F5F90934104909141049F719093F2
:101EF0004104789490E008959091410480914204C7
:101F0000981729F00E94630F482F87FD03C040E017
:101F1000842F0895582F52955F705F30C9F3282F92
:101F200030E02F7030708091AB0490E028173907B3
:101F300071F750933E04ECCF909198048091C000CB
:101F400085FFFCCF906B9093C6008091C00085FF09
:101F5000FCCF8BE78093C6008091C00085FFFCCF4B
:101F60001092C600089580912E04823049F080912D
:101F7000C00085FFFCCF8CEF8093C6000E949C0FB1
:101F80000895909130048913089580E00E94D61C32
:101F90008FEF8093300408951F93182F962F662398
:101FA000B9F060E0809130048F3F09F061E0953630
:101FB00048F4812F895140E00E94BF1C10933004E7
:101FC0001F910895812F895141E00E94BF1CF6CFD7
:101FD00060E00E94C10F1F910895FF920F931F931D
:101FE0008091830581708093830580918305809320
:101FF00070040E94021680918305882309F02EC187
:102000000E9457178BE090E00E94490280932402BF
:102010008CE090E00E94490280932502FF2410E0AA
:102020000E94A6140E94AB28882309F048C0909112
:10203000410480914204981769F00E94630F682F51
:1020400087FD6BC080913E04883009F4ACC08930B4
:1020500009F477C0112371F42091A104222349F4DB
:102060008091AA04882329F480911007882309F419
:10207000E0C010E087E10E943613882389F2809146
:1020800083058F5F809383058091830581708093A2
:102090008305809183058093700480E00E948B15F6
:1020A00080918305882309F4BBCF80E00E945315FB
:1020B0000E94A6140E94AB28882309F4B8CF0E947E
:1020C0009C0F81E0809325068091030780939605FD
:1020D000109226068091C2066091030740911F0668
:1020E0002091250609E616E00E94E72B60911F0665
:1020F000C8010E942029FF2061F08BE090E06091F0
:1021000024020E9450028CE090E0609125020E941F
:1021100050021F910F91FF900895482F42954F70E4
:102120004F3009F498C0282F30E02F703070809124
:10213000AB0490E02817390709F48DC010923E04D3
:102140006FCF67FDBAC0062F0E94630F482F11237F
:1021500009F090CF50912402051748F0852F90E0A8
:102160000F96202F30E0821793070CF082C0509119
:102170002502051708F470CF852F90E00C96202FCC
:1021800030E0821793070CF467CF051B82EA94E0D6
:10219000602F0E94720E8091A2048F778093B10607
:1021A0002091A1045BCF67FD84C0062F0E94630FBE
:1021B000112371F540912402041748F0842F90E018
:1021C0000F96202F30E0821793070CF06BC04091E0
:1021D0002502041708F440CF842F90E00C96202F9E
:1021E00030E0821793070CF437CF041B82EA94E0A7
:1021F000602F0E94CC0E8091AA04882309F42CCF72
:102200008091A2048F778093B1062091A10426CFFC
:10221000113009F456C089E10E948B150093250204
:1022200080918305809370042091A104FF24F3948E
:1022300015CF84E00E9436138823A1F485E00E9424
:102240003613882309F415CF1092700489E10E9497
:10225000531512E00FCF40933E04F4CE80E00E946D
:102260005315CECE1092700480E20E94531511E0F7
:1022700001CF051B89E994E0602F0E94720E209126
:10228000A10420933F04809199048F7780934004A8
:102290008091D804909140048295807F890F80932B
:1022A0004004DCCE041B89E994E0602F0E94CC0E30
:1022B000E6CF0E94630F082F79CF0E94630F082F8B
:1022C00043CF80E20E948B15009324028091830506
:1022D000809370042091A104FF24F394BFCE1F9338
:1022E0000E9417168091AB040E9425160E94A61426
:1022F00084E60E94420E0E94A61484E60E94420ECA
:102300000E94A6148FEF809330040E94A6140E94AE
:10231000AB28882301F590914104809142049817DD
:10232000A1F30E94630F482F87FD19C080913E04DE
:10233000883039F1893049F747FD30C0142F0E94A9
:10234000630F682F812F0E94CC0F0E94A6140E9459
:10235000AB28882301F30E949C0F1F910895582FEA
:1023600052955F705F30B9F0282F30E02F703070D9
:102370008091AB0490E02817390769F010923E0471
:10238000C4CF47FD0FC0142F0E94630F682F812F09
:102390000E94C10FBACF50933E04C8CF0E94630F72
:1023A000182FCDCF0E94630F182FEECF1F920F92E0
:1023B0000FB60F920BB60F9211242F933F934F93AA
:1023C0005F936F937F938F939F93AF93BF93EF939D
:1023D000FF939091C6009A3F09F442C09C3FA9F137
:1023E000983F09F44AC080914204E82FF0E0E45598
:1023F000FB4F90838F5F80934204809142048F71E2
:10240000809342049091420480914104981751F4C2
:10241000809141048F5F80934104809141048F71CA
:1024200080934104FF91EF91BF91AF919F918F9164
:102430007F916F915F914F913F912F910F900BBEC4
:102440000F900FBE0F901F901895809170048823F5
:1024500049F380912E04823029F70E94E32FE2CFC6
:1024600080912E048230F1F680917004882311F05F
:102470000E9424300E948900D5CF809175049091EC
:10248000760490932D0480932C041092760410927D
:10249000750480912E04823029F65C9A8091C000E8
:1024A00085FFFCCF88EF8093C6000E94EC058091E9
:1024B0002C0490912D0496958795909345048093D4
:1024C0004404B0CF80912E04813009F05F980895C4
:1024D00099B1991F9927991F80914604882311F477
:1024E000992321F49093460480E008959093460444
:1024F00081E0089599B1991F9927991F8091470408
:10250000882311F0992321F09093470480E00895E7
:102510001092470481E008958AB1806F8AB98BB127
:102520008F708BB908958AB18F708AB98BB18F7013
:102530008BB9089580912E04882321F45C9881E062
:102540000E94420E5F9A0895AC01F894289800000A
:10255000000000000000289A20E030E01EBC0DB40E
:1025600007FEFDCF8EB5FA01E20FF31F80832F5FC8
:102570003F4F2330310591F77894089516980895C8
:10258000169A089520B1269526952F70822F90E0F7
:102590002695322F369536952270322B880F991F4B
:1025A000282F2470322B880F991F880F991F88704D
:1025B000382B8FE0831B089580B1869586958F70A8
:1025C0000895282F883188F4E82FE695E695E6955A
:1025D000F0E0E752FB4F808190E0277002C09595B4
:1025E00087952A95E2F78170089580E00895282F55
:1025F000883188F4E82FE695E695E695F0E0E0531B
:10260000FB4F808190E0277002C0959587952A95B1
:10261000E2F78170089580E00895282F883188F4CA
:10262000E82FE695E695E695F0E0EC52FB4F8081C9
:1026300090E0277002C0959587952A95E2F7817002
:10264000089580E008958091D904882321F4809131
:10265000DA04882319F090E0892F089590E08091A2
:10266000DB048823C9F791E0892F0895282F88314A
:10267000A0F4482F469546954695277081E090E056
:10268000382F01C0330F2A95EAF7A42FB0E0FD01DF
:10269000E053FB4F8081832319F420E0822F0895BB
:1026A000232F30E020953095A752BB4F8C9190E0BE
:1026B00028233923232B89F7342F3F5F832F63E0AF
:1026C0000E94D745E92FF0E0E752FB4F8081882335
:1026D00021F720E0832F8F5F0E94D745E92FF0E09C
:1026E000E752FB4F80818823C9F621E0D7CF1F93A3
:1026F000CF93DF93C8E3D2E010E088810E94E1121B
:10270000882329F41F5F21961D30B9F71FEF812F11
:10271000DF91CF911F9108951F93CF93DF93C8E36B
:10272000D2E010E088810E94F712882349F41F5FED
:1027300021961D30B9F780E0DF91CF911F91089568
:10274000812F8F5FDF91CF911F9108951F93CF93BA
:10275000DF93C8E3D2E010E088810E940D13882344
:1027600049F41F5F21961D30B9F780E0DF91CF91CA
:102770001F910895812F8F5FDF91CF911F91089551
:102780001F93CF93DF93C0E3D2E010E088810E94D3
:10279000E112882349F41F5F21961830B9F780E0D1
:1027A000DF91CF911F910895812F8F5FDF91CF919E
:1027B0001F9108951F93CF93DF93C0E3D2E010E001
:1027C00088810E94F712882349F41F5F21961830F0
:1027D000B9F780E0DF91CF911F910895812F8F5F2E
:1027E000DF91CF911F9108951F93CF93DF93C0E3A3
:1027F000D2E010E088810E940D13882349F41F5F06
:1028000021961830B9F780E0DF91CF911F9108959C
:10281000812F8F5FDF91CF911F910895CF93DF9329
:10282000C0E3D2E088810E94E112882349F4219616
:1028300082E0C833D807B1F780E0DF91CF910895E7
:1028400081E0DF91CF910895FF920F931F93CF9373
:10285000DF93C0E3D2E0FF2400E006C00F5F2196C3
:1028600082E0C833D80789F01881812F0E94E112D5
:102870008823A1F7812F0E940D13882381F3F394FD
:10288000219682E0C833D80779F781E0F81639F04D
:1028900080E0DF91CF911F910F91FF90089580E02C
:1028A0000730B9F781E0F5CF1F93CF93DF93C6E2EE
:1028B000D2E010E088810E94F712882349F41F5F5C
:1028C00021961A30B9F780E0DF91CF911F910895DA
:1028D000812F8F5FDF91CF911F91089580914904DF
:1028E00010924904089580E00895382F883100F54A
:1028F000282F277081E090E0982F01C0990F2A952A
:10290000EAF7832F869586958695A82FB0E0FD017E
:10291000E053FB4F8081892369F4FD01EC52FB4FAA
:102920008081892371F4A752BB4F8C91982339F48D
:1029300080E00895832F0E94261882E0089583E0A6
:102940000895832F0E942E1881E00895EF92FF9240
:102950000F931F93DF93CF9300D000D0CDB7DEB796
:102960001092D0041092D4041092D1041092D50485
:102970001092D2041092D60480914A048A3068F4EE
:1029800026960FB6F894DEBF0FBECDBFCF91DF9174
:102990001F910F91FF90EF90089510924A0416989E
:1029A0007E010894E11CF11CC7010E94A4128091D1
:1029B000D9048C838091DA048D838091DB048E832B
:1029C00060E070E001E010E0E62FE695E695E69520
:1029D000F0E0CB0187709070980102C0220F331F86
:1029E0008A95E2F7C901AF0147525B4FD701AE0F9D
:1029F000BF1F3C91E452FB4F2081232B282380955D
:102A0000FA0130818323282B20836F5F7F4F683149
:102A10007105D1F60E94C212982F96959093D80412
:102A20008093CE04169A40E050E0BE016C5F7F4F69
:102A3000DA01A452BB4FF701E40FF51F80818C939C
:102A4000FB01E40FF51F2081FA01E752FB4F908153
:102A5000FA01E053FB4F822F809589238083FA018E
:102A6000EC52FB4F9095922390834F5F5F4F433022
:102A70005105F1F690B1969596959F708091CC0492
:102A8000891721F010924B049093CC0480914B0451
:102A90008F3630F09093CD048091CD048093CC0498
:102AA0000E9457176DCF282F8832C0F4E82FE69583
:102AB000E695E695F0E0277081E090E001C0880F90
:102AC0002A95EAF7DF01A45BBB4F2C91282B2C93AE
:102AD000EF5AFB4F80952081822380830895282F11
:102AE0008832C0F4E82FE695E695E695F0E0277089
:102AF00081E090E001C0880F2A95EAF7DF01AF5A24
:102B0000BB4F2C91282B2C93E45BFB4F80952081AD
:102B1000822380830895282F8832C8F4E82FE69511
:102B2000E695E695F0E0277081E090E002C0880F1E
:102B3000991F2A95E2F78095DF01A45BBB4F2C918A
:102B400028232C93EF5AFB4F208182238083089502
:102B5000282F883298F4E82FE695E695E695F0E080
:102B6000EF5AFB4F277081E090E002C0880F991F59
:102B70002A95E2F780952081822380830895282F6B
:102B8000883290F4E82FE695E695E695F0E0E45B70
:102B9000FB4F277081E090E002C0880F991F2A95B3
:102BA000E2F72081282720830895E82F883298F4BF
:102BB000282F277081E090E002C0880F991F2A9586
:102BC000E2F7E695E695E695F0E0EF5AFB4F2081B7
:102BD0002823822F089520E0822F0895982F96951C
:102BE00096959695ECE4F4E0E90FF11D208130E034
:102BF000877002C0359527958A95E2F7217030706D
:102C0000C90108951092500410924F0410924E047E
:102C100010924D0410924C041092550410925404DA
:102C20001092530410925204109251040895CF93BD
:102C3000DF93C4EAD2E089910E948B1582E0C43B05
:102C4000D807C9F7DF91CF910895803108F0089532
:102C5000E82FF0E0EC55FD4F80810E945315089558
:102C60000F931F93CF93DF93082FC4EAD2E010E0B5
:102C700007C088810E9453151F5F2196103149F0CB
:102C80001017B8F388810E948B151F5F21961031B1
:102C9000B9F7DF91CF911F910F910895803108F01E
:102CA0000895E82FF0E0EC55FD4F80810E946F15EC
:102CB0000895803110F080E00895E82FF0E0EC55A1
:102CC000FD4F80810E94EE150895803110F080E064
:102CD0000895E82FF0E0EC55FD4F80810E94D51556
:102CE0000895883108F00895E82FF0E0E158FD4F8D
:102CF00080810E9453150895883108F00895E82FC7
:102D0000F0E0E158FD4F80810E946F1508958831F1
:102D100008F00895E82FF0E0E158FD4F80810E940F
:102D20008B150895CF93DF93CFE7D2E089910E946E
:102D30008B1582E0C739D807C9F7DF91CF91089585
:102D4000E82F8150883008F00895F0E0EA58FD4FF0
:102D500080810E94531508950F931F93CF93DF93A3
:102D6000082FC7E7D2E011E007C088810E948B15C9
:102D70001F5F2196193069F01017B9F7E12FF0E0C5
:102D8000EA58FD4F80810E9453151F5F219619302C
:102D900099F7DF91CF911F910F910895E82F8150FE
:102DA000883008F00895F0E0EA58FD4F80810E94D5
:102DB0008B150895E82F8150883008F00895F0E0D1
:102DC000EA58FD4F80810E946F150895E82F8150C9
:102DD000883010F080E00895F0E0EA58FD4F8081DF
:102DE0000E94D5150895E82F8150883010F080E0BA
:102DF0000895F0E0EA58FD4F80810E94EE15089595
:102E0000CF93DF93C7E7D2E089910E948B1582E0D0
:102E1000CF37D807C9F7DF91CF9108958D3008F0EB
:102E20000895E82FF0E0E956FD4F80810E94531588
:102E300008958D3008F00895E82FF0E0E956FD4F31
:102E400080810E948B1508958D3008F00895E82F39
:102E5000F0E0E956FD4F80810E946F150895E7E983
:102E6000F2E0E80FF11D80810E94D5150895CF93FF
:102E7000DF93C7E9D2E089910E948B1582E0C43AC2
:102E8000D807C9F7DF91CF9108950E94371784E0E2
:102E90000E948B1583E00E948B1588E00E948B15A1
:102EA00081E00E948B1582E00E948B150895F894B2
:102EB000179820E030E090915604F901EF5AFB4F4B
:102EC00080819823F901E45BFB4F8081982B9EBDA4
:102ED0000DB407FEFDCF2F5F3F4F2530310559F769
:102EE000179A78940895ECE4F4E0A1E5B4E08081C9
:102EF0009D91892B819384E0E135F807C1F708950E
:102F0000ECE4F4E0A1E5B4E09D9190958081892303
:102F1000819384E0E135F807B9F70895ECE4F4E033
:102F2000A1E5B4E020819C91892F822319F090952E
:102F3000922390831D92319684E0E135F80791F752
:102F400008951F93182F84E00E948B15123049F0CA
:102F500083E00E948B15113071F01F3F39F01F91F3
:102F6000089583E00E946F151F91089584E00E94E8
:102F700053151F91089583E00E9453151F910895E2
:102F80000F931F93CF93DF93182F87FD50C086E1D7
:102F90000E948716812F829586958695837080FF83
:102FA00029C085E10E9471161F7349F11731A0F500
:102FB0008FEF0E94A11784E10E948716012F10E075
:102FC000CBE0D0E0C017D10731F0FE01E457FD4F50
:102FD00080810E948B152196C831D10599F704573D
:102FE0001D4FF80180810E945315DF91CF911F91F1
:102FF0000F91089585E10E9487161F73B9F680E04E
:103000000E94A1170E94371784E10E947116DF9178
:10301000CF911F910F910895143268F0103370F41E
:10302000185181E00E94A117112329F6EBCF86E108
:103030000E947116AFCF1C5080E0F4CF1C3318F4FF
:10304000145282E0EFCF105383E0ECCFEFE7F2E0D1
:10305000E80FF11D80810E9453150895EFE7F2E01B
:10306000E80FF11D80810E948B150895E7E7F2E0DB
:10307000E80FF11D80810E9453150895E7E7F2E003
:10308000E80FF11D80810E948B150895DF92EF9269
:10309000FF920F931F93CF93DF93F02EDE2C22230A
:1030A00071F1022F040FE42EC7E7D2E010E00BC04D
:1030B000101758F41F15D9F088810E9453151F5F0F
:1030C0002196183049F01E1598F788810E948B15BB
:1030D0001F5F21961830B9F781E08D15A0F4DF91BC
:1030E000CF911F910F91FF90EF90DF900895E12F06
:1030F000F0E0E958FD4F80810E946F15E0CF062F68
:10310000080FE82ED1CFDD2071F088E00E948B15EA
:1031100081E00E945315DF91CF911F910F91FF9095
:10312000EF90DF90089588E00E94531581E00E949F
:103130008B15DF91CF911F910F91FF90EF90DF9052
:103140000895FF920F931F93082FF62E84E00E949C
:103150008B1583E00E948B1588E00E948B1581E01F
:103160000E948B15102F04FD34C015FD29C007FDEA
:103170002CC016FD21C00E943717FF2099F0802F28
:103180008F708D3098F08BE10E9453158CE10E9476
:1031900053158FE00E9453158EE00E9453158DE069
:1031A0000E9453151F910F91FF9008950E940E17D2
:1031B0001F910F91FF90089581E00E945315DBCF7E
:1031C00083E00E94531507FFD4CF88E00E94531577
:1031D000D0CF84E00E945315C8CFE5E4F2E0E80FB9
:1031E000F11D808108958A3008F00895E82FF0E0FD
:1031F000E359FD4F80810E9453150895CF93DF93CB
:10320000CDE6D2E089910E948B1582E0C737D807BE
:10321000C9F7DF91CF91089590914C04982790932E
:103220004C0490914D04982790934D0490914E0436
:10323000982790934E0490914F04982790934F04B1
:10324000909150049827909350040895AC01611513
:103250007105A1F020E0E0E0A0E0B0E0A40FB51F10
:103260008C91E827F0E0E454FD4FE0812F5FA22F1E
:10327000B0E0A617B70790F38E2F0895E0E0FCCFDB
:103280000E94A6140E94AB288823D1F30895EF92E0
:10329000FF920F931F93CF93DF937C018B016115F6
:1032A000710561F0C0E0D0E0F701EC0FFD1F8081F7
:1032B0000E94CE012196C017D107B0F3DF91CF91C4
:1032C0001F910F91FF90EF90089522E42093DF0467
:1032D0001092E00422E02093E1049093E2048093B2
:1032E000E304AFEDB4E0E0E08D91E827F0E0E454D2
:1032F000FD4FE08184E0A43EB807B1F7EC93CD0127
:10330000059766E070E00E944719089590E8909351
:10331000DF041092E00421E02093E1048093E204B2
:10332000ACEBB2E090913C03FD01E90FF11D9081FF
:103330009227FD01E90FF11D90819827A90FB11D7A
:103340008C918093E3048FED94E065E070E00E943F
:10335000471908951F920F920FB60F920BB60F9256
:103360001124DF92EF92FF920F931F932F933F93BD
:103370004F935F936F937F938F939F93AF93BF937D
:10338000CF93DF93EF93FF931091CE008091BB0218
:10339000882309F46EC08091590490915A04895E83
:1033A000934008F080C080915704803408F089C0B1
:1033B000282F2F5FE82FF0E0E15EFA4F1083209373
:1033C000570410925A0410925904233008F451C043
:1033D00070911F059091200580E060912105462F96
:1033E00050E0482B592B30E0CA01049628173907C2
:1033F00008F43FC09A012D5F3F4FF901E15EFA4F9B
:1034000010812115310509F401C190E0E0E0A0E050
:10341000B0E0A15EBA4F8C91E827F0E0E454FD4F94
:10342000E0819F5FA92FB0E0A217B30790F31E17AA
:1034300009F450C02115310509F4EAC090E0E0E03C
:10344000A0E0B0E0A15EBA4F8C91E827F0E0E45430
:10345000FD4FE0819F5FA92FB0E0A217B30790F363
:103460008E2F90E00E94AA011092570480E00E94E3
:103470008619FF91EF91DF91CF91BF91AF919F910D
:103480008F917F916F915F914F913F912F911F91FC
:103490000F91FF90EF90DF900F900BBE0F900FBE3B
:1034A0000F901F9018950E9417160E94571710939F
:1034B0001F0581E08093570410925A04109259041A
:1034C000D8CF0E9486191092570410925A04109275
:1034D0005904CFCF713809F492C17238B0F5713107
:1034E00009F42BC1723108F096C0713051F170317E
:1034F00031F080E00E94861910925704BACF6231F1
:10350000C1F780912205082F10E0000F111F000F56
:10351000111F000F111F80912305080F111D029527
:103520001295107F1027007F1027C4E2D5E0899103
:10353000B8010E949D1D0F5F1F4F85E0C433D8075F
:10354000B1F781E00E948619D7CF763809F435C1EA
:10355000773808F073C0723809F484C1753849F6B9
:103560004330510509F0A5C030912205932F80E02A
:1035700020912305E22EFF24E82AF92AD090240581
:10358000EAE3ED1508F4B6CF7093DF041092E0047F
:10359000F2E0DF0ED092E1048EEFD80E3093E20419
:1035A0002093E304DD2071F004EE14E0E701CE0186
:1035B0000E94E11DF80181938F0121969E012E1931
:1035C0002D15A8F38091E104682F6D5F09F4D5C132
:1035D000AFEDB4E090E08E5F282F30E020523B4FFB
:1035E0008D919827E92FF0E0E454FD4F9081A217C8
:1035F000B307B1F7E62FF0E0E152FB4F90836F5F26
:103600008FED94E070E00E94471976CFE0E00FCF95
:1036100080E090E027CF703409F453C1713409F091
:1036200068CF623009F065CF9091220580E020914B
:103630002305820F911D0E94B4025ECF7738E9F115
:10364000783809F056CF7093DF041092E00480912F
:103650002205813009F46AC1813008F05BC180E144
:103660008093E2041092E3048093E4041092E50452
:1036700084E047E0A7E0B0E068E070E08093E10418
:1036800090E020E030E0F901E152FB4F8081982783
:10369000E92FF0E0E454FD4F90812F5F3F4F241756
:1036A00090F3A152BB4F9C938FED94E00E94471979
:1036B00023CF80E00E9486191FCF809122058823A6
:1036C00009F006C14230510509F014CFE0912305FD
:1036D000E43008F00ECF89E18093DF041092E0041B
:1036E00080E18093E1042E2F30E022953295307FE7
:1036F0003227207F3227A2EEB4E0F901E759F94FD3
:1037000080818D932F5F3F4F84E0A23FB807A9F7D8
:103710005397E0E08D91E827F0E0E454FD4FE0811D
:10372000F4E0A23FBF07B1F7E093F204CD01439765
:1037300064E170E00E944719DFCE623009F0D9CE13
:1037400080912205082F10E0000F111F000F111F9C
:10375000000F111F80912305080F111D029512956E
:10376000107F1027007F102789E18093DF041092DB
:10377000E00480E18093E104C2EED4E0C8010E943D
:10378000E11D89930F5F1F4F34E0C23FD307B1F7AC
:10379000DE015397E0E08D91E827F0E0E454FD4F1F
:1037A000E081CA17DB07B9F7E093F2048FED94E0EC
:1037B00064E170E00E9447199FCE9091220580E05D
:1037C00020912305E22EFF24E82AF92A2EEFD22E9B
:1037D000D60E63506A3308F06CCFDD2009F4B1CE09
:1037E00004E215E0E701F80181918F01BE010E941A
:1037F0009D1D21969E012E192D15A8F3A2CE87E1BD
:1038000090E09093E3048093E2048CEC90E090933A
:10381000E5048093E404E4EBF2E0A6EEB4E08191E9
:103820008D9322E0EA3BF207D1F781E88093DF0431
:103830001092E0048AE08093E104AFEDB4E0E0E0B0
:103840008D91E827F0E0E454FD4FE08134E0AC3E98
:10385000B307B1F7EC93CD010D976EE070E00E94D5
:1038600047194ACE4230510509F023CF3091220545
:10387000332309F468C09091230520E082E8809307
:10388000DF041092E00483E08093E1043093E204CB
:103890009093E3042093E404AFEDB4E0E0E08D9175
:1038A000E827F0E0E454FD4FE08184E0A53EB8074E
:1038B000B1F7EC93CD01069767E070E00E944719DD
:1038C0001BCE80917A0490917B040E94651914CEDE
:1038D000813009F00ECE4231510509F00ACEE09157
:1038E0002305E43008F005CE2E2F30E0A4E2B5E049
:1038F00022953295307F3227207F32278D91F90132
:10390000E759F94F80832F5F3F4F85E0A433B80715
:10391000A9F717CE883009F0ECCD81E08093E2045E
:1039200044E0A4E0B0E065E070E0A8CE88E08093D9
:10393000E20480E18093E30482E045E0A5E0B0E0AA
:1039400066E070E09BCE90912305973860F495383F
:1039500070F4993181F0993120F0892F81588230AB
:1039600030F020E08BCF973821F09838D1F721E064
:1039700085CF24E083CF20E181CF90E03BCE2C980F
:10398000803408F08FE3611160E4442349F090E053
:10399000882349F0682B962B98B92C9A2D9A089574
:1039A00090E88823B9F7962B98B90895882319F4DD
:1039B0002D982C980895469A2C9808959F92AF922E
:1039C000BF92CF92DF92EF92FF920F931F93CF930C
:1039D000DF930E941716809198040E9425160E947A
:1039E000A6140E946E14BB249924AA24CC240E94FD
:1039F000A6140E94AB28882309F073C02B2D3CE04D
:103A00002302C001112497E1D92ED80EEA2CE294AA
:103A1000EE0CEE0C80ECE822C0E0D0E009C0802F74
:103A20000E940D13882319F52196CD30D10559F147
:103A3000FC2EFE01E454FC4F0081802F0E94F712FF
:103A4000882369F31C2F1D0D812F6C2D4A2D0E9498
:103A5000BF1C812F8E290E94010F8C2F0E940E17F0
:103A6000CC24C394802F0E940D138823E9F28F2D5C
:103A70008D0D8E290E94270F8F2D0E9419172196D8
:103A8000CD30D105A9F68FE00E94F712882309F402
:103A900042C081E08B150CF04EC09B1429F08B2D99
:103AA0000E94A1170E94571784E10E94F7128823F1
:103AB00051F080E0AA2009F481E0A82E8823B9F112
:103AC00088E00E94531586B190E08F739070892B27
:103AD000B1F49B2C0E94A6140E94AB28882309F401
:103AE0008DCF0E949C0FDF91CF911F910F91FF907E
:103AF000EF90DF90CF90BF90AF909F9008950E947D
:103B00002313882331F380E00E94D61C0E943717CC
:103B1000CC249B2CDFCF8EE00E94F712882309F47F
:103B2000BCCF2FEFB21609F4B8CFBA94B6CF88E065
:103B30000E948B15C8CFB394B0CF282FF89495E08E
:103B4000289800000000000000009EBD0DB407FE94
:103B5000FDCF00000000000000001EBC0DB407FEF9
:103B6000FDCF8EB5289A000000000000000080FD07
:103B7000E7CF28980000000086E08EBD0DB407FE58
:103B8000FDCF00000000289A0000000000000000A7
:103B900028980000000082E08EBD0DB407FEFDCF26
:103BA0007EBD0DB407FEFDCF6EBD0DB407FEFDCF8B
:103BB0002EBD0DB407FEFDCF00000000289A7894BA
:103BC0000895382FF89425E02898000000000000A0
:103BD00000002EBD0DB407FEFDCF00000000000068
:103BE00000001EBC0DB407FEFDCF8EB5289A000064
:103BF00000000000000080FDE7CF289800000000D2
:103C000083E08EBD0DB407FEFDCF9EBD0DB407FE53
:103C1000FDCF3EBD0DB407FEFDCF000000001EBC71
:103C20000DB407FEFDCF8EB5289A78940895892F9C
:103C30008F7184FD806E0895EF92FF920F931F9312
:103C4000FA01D90186958083862F90E08F7090705D
:103C50009595879595958795959587958C93862FBE
:103C60008770F801808362956F70F70160831F9100
:103C70000F91FF90EF900895FC0130E0229532956E
:103C8000307F3227207F322720838081660F660FA6
:103C9000660F640F6F70862B8083089580915B049C
:103CA000882349F087FD0EC083E00E94531584E00D
:103CB0000E948B15089583E00E948B1584E00E947A
:103CC0008B15089583E00E948B1584E00E945315A4
:103CD0000895962F803110F08FEF0895682F70E0CF
:103CE000660F771F6F5F734F892F0E949D1D80E0C5
:103CF00008959B01803120F5682F70E0FB01EE0FE5
:103D0000FF1FE753FC4F8081918128173907A0F0EE
:103D1000009749F08150660F771F6050744F0E94E2
:103D20009D1D80E0089580E0660F771F6050744FFE
:103D30000E949D1D80E00895C901009759F7F3CFB7
:103D40008FEF0895803198F470E06050784F90E0E4
:103D50000024969587950794969587950794982FB4
:103D6000802D680F791F8CE06030780710F08FEF9E
:103D70000895842F0E949D1D80E00895EF92FF9288
:103D80000F931F93CF93DF93C82FD0E0CC0FDD1F8D
:103D9000CC0FDD1FCC0FDD1FC60FD11DC05CDF4F68
:103DA000CC0FDD1FC295D295D07FDC27C07FDC27EA
:103DB000EE24FF248701000F111F015A1A4FF8014A
:103DC00080819181892FBE010E949D1DF801808113
:103DD00091812196BE010E949D1D0894E11CF11C59
:103DE0002196F0E1EF16F10429F7DF91CF911F91B1
:103DF0000F91FF90EF90089590E0880F991F8F5FCB
:103E0000934F0E94E11D90E008950F931F93082F98
:103E100010E0000F111FC8018050944F0E94E11D57
:103E200090E0019607531C4FF801208131818217E1
:103E3000930708F49C01C9011F910F910895809187
:103E4000CE0480939005809190050E94051F909369
:103E50008B0580938A05809190050E94FC1E9093AB
:103E60009205809391052091910530919205809162
:103E70008A0590918B052817390720F0109292053A
:103E80001092910580917F0590918005E0919005B9
:103E9000F0E0EE0FFF1FE753FC4F608171810E943D
:103EA000E3459093800580937F050895803198F4D1
:103EB00070E06050784F90E00024969587950794C5
:103EC000969587950794982F802D680F791F8CE021
:103ED0006030780710F08FEF0895CB010E94E11D4C
:103EE0000895EF92FF920F931F93CF93DF93E0908B
:103EF0007F05F09080050894E11CF11C80E00E9491
:103F000036138823C9F400E080919305813029F1AC
:103F100080E00E940D13882329F080919305882367
:103F200009F0BFC0013009F4E7C0DF91CF911F91C4
:103F30000F91FF90EF90089581E080939305109288
:103F40008F0510928E058093620482E20E948B1589
:103F500001E0809193058130D9F60E945414282FF6
:103F60008823B9F0215080918E0590918F057C01B6
:103F7000EE0CFF1CEE0CFF1CEE0CFF1C880F991FB3
:103F8000E80EF91EE20EF11CF0928F05E0928E050C
:103F900001E087E10E94F712882341F0E09091054B
:103FA000F09092050894E11CF11C01E083E00E946E
:103FB000F712882329F0E0908A05F0908B0501E044
:103FC00089E00E94F712882309F0A2C089E00E94CC
:103FD0000D13882309F0BAC08AE00E94F7128823E3
:103FE00009F0A5C08AE00E940D13882309F490CF40
:103FF0008CE10E948B15E091900520918A0530910B
:104000008B05F0E0EE0FFF1FE753FC4F808191819D
:104010002817390708F07CCF80918A0590918B058D
:10402000019690938B0580938A058091900560910D
:104030008A0570918B050E94791E809190050E94DF
:10404000051F90938B0580938A0560918A05709176
:104050008B056150704080917F0590918005861797
:104060009707D8F4EB01219701C0E90180919005F1
:104070001C2F6C2F0E94561F482F809190051F5FA8
:10408000612F0E94A21E9E012150304080917F0529
:10409000909180058C179D0740F388E0809365041C
:1040A00037CF82E20E94531510926204109293055A
:1040B00081E08093650420918E0530918F05211554
:1040C0003105A9F0E0919005F0E0EE0FFF1FE753F6
:1040D000FC4F808191818217930748F02150304036
:1040E0003093800520937F0587E0809365041092CC
:1040F0003804013009F019CFC7010E94EB01009389
:104100003804DF91CF911F910F91FF90EF900895A8
:104110008BE10E94531510928F0510928E05E0904E
:104120007F05F09080050894E11CF11C4FCF8CE1D5
:104130000E94531510928F0510928E05E0907F0516
:10414000F09080050894E11CF11C4CCF8BE10E949B
:104150008B15C0917F05D0918005219680918A05AD
:1041600090918B05C817D90708F036CF809190053C
:104170001C2F6C2F0E94561F482F809190051150C4
:10418000612F0E94A21E219680918A0590918B0535
:10419000C817D90758F380918A0590918B0501972C
:1041A00090938B0580938A058091900560918A0594
:1041B00070918B050E94791E809190050E94051FC9
:1041C00090938B0580938A0588E08093650404CFE3
:1041D000EF92FF920F931F938091CE0480939005EE
:1041E000809190050E94051F90938B0580938A050E
:1041F000809190050E94FC1E9093920580939105FA
:10420000209191053091920580918A0590918B05BE
:104210002817390720F0109292051092910580918D
:104220007F0590918005E0919005F0E0EE0FFF1F73
:10423000E753FC4F608171810E94E34590938005B4
:1042400080937F058091900560917F057091800536
:104250000E94561F80938705809190056091870585
:104260004EED55E026E935E008E915E0EAEAEE2EE4
:10427000E6E0FE2E0E941C1E81E0809326060E942E
:10428000DC288091AA068093B1061F910F91FF90C0
:10429000EF900895AF92BF92CF92DF92EF92FF928C
:1042A0000F931F93CF93DF93C82EDD24CC0CDD1C1E
:1042B000CC0CDD1CCC0CDD1CC60ED11C80E490E0C7
:1042C000C80ED91ECC0CDD1CC294D29410EFD122A2
:1042D000DC24C122DC24AA24BB24C6010E94E11DE7
:1042E000D82FC0E07501EE0CFF1CEFE5F5E0EE0EF7
:1042F000FF1EF701D183C08300811181C6010196A1
:104300000E94E11D90E0082B192BF7011183008317
:104310000894A11CB11C82E090E0C80ED91E90E167
:10432000A916B104D1F6DF91CF911F910F91FF90A3
:10433000EF90DF90CF90BF90AF90089510928905D5
:1043400084E20E948B150E9402160E948E17109222
:10435000240680E00E94D61C0895109288051092D1
:1043600024061092810580E00E94D61C0E9402164D
:104370000E948E170E946E14089580918505909179
:104380008605682F6770969587959695879596957B
:1043900087958F700E94A92C609185057091860584
:1043A0009B0140E050E0DA01C90180709078A07074
:1043B000B070892F9A2FAB2FBB2780936C04DA0142
:1043C000C90180709074A070B070892F9A2FAB2FA4
:1043D000BB2780936A042070307240705070232F86
:1043E000342F452F552720936B0410929905872F62
:1043F0008F7184FD806E089581E08093880581E24D
:104400000E94531510926A0480916A0480936B0491
:1044100080916B0480936C041092810510922406A5
:1044200080915F0590916005909386058093850546
:104430008F5F9F4F89F010928D0510929905109211
:1044400078040E94BD2180935B0480912F0480FD3D
:10445000FCCF81E0809381050E941716089581E0CA
:104460008093890584E20E9453150E9417160895CF
:10447000DF92EF92FF920F931F9380911007882392
:1044800009F483C284E00E9460291092840580911F
:104490008405809383051092930510928F051092E6
:1044A0008E050E94E8208091C2066091030740912A
:1044B0001F062091250609E616E00E94E72B809151
:1044C0001F066091250640919805209126060091CF
:1044D0009C05E09096050E94461857E0D52E07C02F
:1044E000113009F4FBC00E947E2B8823C9F00E9482
:1044F000A6141091A9061330D9F0143088F31430A3
:10450000D9F11D3081F781E00E946F308091A906BA
:104510008D3049F3109270040E947E2B882339F766
:104520000E944D2B0E94A6141091A906133029F762
:104530000E946629882309F09EC10E94D82A8823F8
:1045400021F010926204109270040E948C13882350
:1045500051F2182F11500E943717812F0E940E1709
:104560001093AA0680911007882309F0BCCF809190
:10457000AA068093B106B7CF0E946629882309F066
:104580005CC180919305882309F44AC10E94711F80
:1045900083E00E943613882309F03BC187E10E9423
:1045A0003613882309F02EC186E10E943613882332
:1045B00009F468C080912606882309F0B0C1809173
:1045C000AA068093B106E0907F05F0908005809167
:1045D0008405882309F090C180912506882309F479
:1045E0004AC010E02091030730911F068091B10668
:1045F00090E082959295907F9827807F982780936E
:10460000870580918705220F220F220F230F210F8C
:104610002F70282B209387058091900560917F054E
:1046200070918005409187050E94A21E1F5F8091B6
:104630007F059091800501969093800580937F057A
:104640000894E11CF11C80917F0590918005E09118
:104650009005F0E0EE0FFF1FE753FC4F6081718182
:104660000E94E3459093800580937F058091250605
:10467000181708F4B7CF80918305882309F052C139
:10468000D092650480916504873009F407C1809158
:104690006504883009F459C180916504813009F4BA
:1046A000AEC08091A906843011F010927004809100
:1046B0001007882309F4DBC080916F04813009F072
:1046C00012CF10926F040E94AB28882309F40BCFFD
:1046D0001F910F91FF90EF90DF9008950E9466293F
:1046E000882309F073C00E94711F83E00E94361373
:1046F000882339F583E00E940D138823F1F490910B
:1047000090058091CE04981711F00E94E8208091C6
:10471000A906813011F0109270048091100788234F
:1047200009F0B8C00E94AB28882309F4DCCE1F91A1
:104730000F91FF90EF90DF90089583E20E948B1518
:10474000DECF1092800510927F05809190056091D8
:104750007F05709180050E94561F80938705809188
:104760009005609187054EED55E026E935E008E9B2
:1047700015E0AAEAEA2EA6E0FA2E0E941C1E81E0AD
:10478000809326068091AA068093B1060E94DC28B9
:104790008091C2066091030740911F062091250673
:1047A00009E616E00E94E72B80911F06609125061E
:1047B000409198052091260600919C05E090960571
:1047C0000E94461883E20E94531594CF0E9402165D
:1047D00082E20E9453151093700481E20E948B15AF
:1047E00080911F066091250640919805209126062C
:1047F00000911F06E09096050E94461874CF109213
:1048000065044FCF81E08093840580E00E946F159E
:10481000CBCE81E08093830583E20E946F15BECEEC
:104820000E946B2B9091900596959093D8048823C5
:1048300009F0ACCE0E946F30A9CE0E94021682E22F
:104840000E94531581E08093700481E20E94531509
:1048500080911F06609125064091980520912606BB
:1048600000911F06E09096050E9446188ACE81E0CE
:104870000E94602921CF0E94021611E01093620469
:1048800084E20E9453158091AA060E940E1710938D
:10489000700453CE84E00E94602944CF809190053B
:1048A00060917F05709180050E94561F8093870557
:1048B00080919005609187054EED55E026E935E041
:1048C00008E915E09AEAE92E96E0F92E0E941C1EEE
:1048D00011E01093260680911F06609125064091F5
:1048E00098052091260600919C05E09096050E946F
:1048F000461810936504D0CE1092840580919005DF
:104900006E2D0E94691E809190050E94FC1E90935E
:1049100092058093910580E00E948B155DCE0E94E8
:10492000DC284DCE1092830580919005B7010E943E
:10493000791E809190050E94051F90938B058093AE
:104940008A0583E20E948B159BCE80919005609131
:104950007F05709180050E94561F80938705809186
:104960009005609187054EED55E026E935E008E9B0
:1049700015E0BAEAEB2EB6E0FB2E0E941C1E81E089
:10498000809326061092650487CE81E00E946029FC
:104990007CCDEF92FF920F931F9380911007882395
:1049A00009F4AAC184E00E946029109284058091D4
:1049B0008405809383051092930510928F051092C1
:1049C0008E050E94E8208091C20660910307409105
:1049D0001F062091250609E616E00E94E72B80912C
:1049E0001F066091250640919805209126060091AA
:1049F0009C05E09096050E94461808C0143009F402
:104A00005FC00E947E2B882309F490C00E94A614E8
:104A10001091A906113091F70E946629882309F0A8
:104A2000DAC083E00E943613882309F0F5C083E0E2
:104A30000E940D13882309F039C180E00E943613CB
:104A4000882309F03CC180E00E940D13882309F0FF
:104A50004BC1909190058091CE049817E1F00E948F
:104A6000E8208091C2066091030740911F062091C3
:104A7000250609E616E00E94E72B80911F0660914B
:104A80002506409198052091260600919C05E0900E
:104A900096050E9446188091A906813011F0109267
:104AA000700480911007882309F043C00E94AB284E
:104AB000882309F4A6CF1F910F91FF90EF900895DE
:104AC0000E946629882309F065C086E10E9436139A
:104AD000882309F053C083E00E943613882309F02D
:104AE00041C080E00E943613882339F580E00E949F
:104AF0000D13882379F58091A906843011F0109266
:104B0000700480911007882309F461C080916F04BC
:104B1000813009F076CF10926F040E94AB28882371
:104B200051F60E947E2B882309F070CF0E944D2BF6
:104B30006DCF84E00E946029B9CF11E010939305F6
:104B400082E20E948B151093380480E00E940D13BE
:104B5000882389F282E20E945315109293051092E5
:104B60003804C9CF81E08093830583E20E94531506
:104B70001092840580E00E948B15B3CF81E0809372
:104B8000840580E00E9453151092830583E20E9401
:104B90008B15A1CF0E94021682E20E94531581E07C
:104BA0008093700481E20E94531580911F066091EA
:104BB0002506409198052091260600911F06E09059
:104BC00096050E94461881E00E9427027ECF81E070
:104BD0000E9460299BCF0E94021682E20E94531518
:104BE0001093700481E20E948B1580911F066091E2
:104BF0002506409198052091260600911F06E09019
:104C000096050E94461881E00E94270283E00E94D8
:104C10003613882309F40BCF1092800510927F057C
:104C20008091900560917F05709180050E94561FCC
:104C30008093870580919005609187054EED55E042
:104C400026E935E008E915E07AEAE72E76E0F72E66
:104C50000E941C1E81E0809326068091AA06809304
:104C6000B1060E94DC288091C20660910307409142
:104C70001F062091250609E616E00E94E72B809189
:104C80001F06609125064091980520912606009107
:104C90009C05E09096050E94461883E20E945315F9
:104CA00083E00E940D13882309F4C7CE83E20E949B
:104CB0008B1580E00E943613882309F4C4CE11E0DE
:104CC0001093930582E20E948B1580917F0590914D
:104CD000800501960E94EB011093380480E00E9449
:104CE0000D13882309F4B5CE82E20E945315109269
:104CF000930510923804ADCE81E00E94602955CE14
:104D0000EF920F931F9310925D04809110078823F8
:104D100009F41DC284E00E946029109284058091EC
:104D20008405809383051092930510928F0510924D
:104D30008E050E941F1F07C0113009F48FC00E940A
:104D40007E2B8823C9F00E94A6141091A906133067
:104D5000D9F0143088F31430D9F11D3081F781E097
:104D60000E946F308091A9068D3049F31092700433
:104D70000E947E2B882339F70E944D2B0E94A61497
:104D80001091A906133029F70E946629882309F09B
:104D9000B0C00E94D82A882321F010926204109299
:104DA00070040E948C13882351F2182F11500E9416
:104DB0003717812F0E940E171093AA0680911007B3
:104DC000882309F0BCCF8091AA068093B106B7CFA3
:104DD0000E946629882309F0D5C080919305882315
:104DE00009F4C3C083E00E943613882329F0809120
:104DF0005D04813009F487C187E10E94361388235E
:104E000009F08CC080E00E943613882309F092C01C
:104E100080E00E940D13882309F09AC08091A906B2
:104E2000843011F01092700480911007882309F4E7
:104E30006FC080916F04813009F081CF10926F04B0
:104E400080915D04882309F07ACF0E94AB288823E3
:104E500009F475CF1F910F91EF9008950E94662974
:104E6000882309F0D9C080919305882309F4F9C0FB
:104E700083E00E943613882379F081E080935D04FB
:104E800080915D04882309F432C183E20E945315A6
:104E90001092800510927F0580E00E9436138823CF
:104EA00009F0ECC010919305113009F4FFC080E0C7
:104EB0000E940D13882309F089C09091900580917C
:104EC000CE04981711F00E941F1F8091A90681300F
:104ED00011F01092700480911007882309F4B5CF67
:104EE00084E00E9460290E94AB28882309F427CF20
:104EF000B1CF0E94021611E01093620484E20E9476
:104F000053158091AA060E940E171093700441CF8A
:104F100081E00E94602910925D048BCF81E0809334
:104F2000840580E00E946F1580E00E94361388237C
:104F300009F46ECF11E01093930582E20E948B1565
:104F40001093380480E00E940D13882309F466CF83
:104F500082E20E94531510929305809138048130AB
:104F600009F4E6C01092380459CF0E946B2B90913F
:104F7000900596959093D804882309F033CF0E942A
:104F80006F3030CF0E94021682E20E94531581E0FA
:104F90008093700481E20E94531580911F066091F6
:104FA0002506409198052091260600911F06E09065
:104FB00096050E94461880915D04882309F49BC0E1
:104FC00083E20E946F150E94571707CF82E20E946A
:104FD00053151092930520918E0530918F05211560
:104FE000310591F0E0919005F0E0EE0FFF1FE753DF
:104FF000FC4F808191818217930730F0215030401F
:105000003093800520937F0580913804813009F426
:1050100080C01092380451CF0E94021682E20E9492
:1050200053151093700481E20E948B1580911F0626
:1050300060912506409198052091260600911F0653
:10504000E09096050E94461880915D04882309F43B
:1050500056C083E20E94531580919305882309F07E
:1050600007CF0E946B2B9091900596959093D80452
:10507000882309F0FDCE0E946F30FACE11E0109324
:10508000930510928F0510928E0582E20E948B1577
:1050900080917F059091800501960E94EB0110930D
:1050A000380410919305113009F001CF0E94541477
:1050B000482F882309F4FBCE415020918E05309172
:1050C0008F05C901880F991F880F991F880F991F95
:1050D000220F331F820F931F840F911D90938F0512
:1050E00080938E050E94EB0110933804E0CE83E29A
:1050F0000E948B15CDCE83E20E948B1564CF83E294
:105100000E948B15B0CE8093830583E20E945315D5
:1051100073CE80911F0660912506409198052091DD
:10512000260600911F06E09096050E94461871CF52
:1051300080911F06609125064091980520912606D2
:1051400000911F06E09096050E9446180BCF81E063
:105150000E946029E2CD9091CD048091D3048917FB
:1051600031F08091CD048093D30481E0089580E0F4
:10517000089580912606882391F08091DE05809322
:10518000C2068091960580930307809198058093CD
:105190001F06809126068093250610922606809190
:1051A0002506882329F080912506809325060895F9
:1051B00081E08093250608958091DE058093C206E4
:1051C00080919605809303078091980580931F0630
:1051D0008091260680932506109226060895833036
:1051E00059F0843050F0843029F08091AA068093E1
:1051F000B10608951092AA0608958230B0F7089576
:10520000FC0187858F708D30C1F030E020E190E0A7
:1052100080818F708E3061F09F5F31969217C0F35E
:10522000892F913118F48150832B089580E1FBCFB1
:105230009923B1F780E0832B089530E12FE0E7CF89
:105240001F93DF93CF930F92CDB7DEB7162F0E9437
:105250000029898389818F708F5F8093EB0310937E
:105260009C05898184FD08C086E08093E9030F9046
:10527000CF91DF911F91089588E08093E9030F900B
:10528000CF91DF911F910895E82FF0E0EF73F07058
:10529000E451FC4F8081089540939A056093DD05A9
:1052A0008093A90681E0809322060895882339F02F
:1052B0008091DD058093A90681E080932206089500
:1052C0008093A90681E080932206089580912206AA
:1052D000882319F01092220681E008953F924F92A0
:1052E0005F926F927F928F929F92AF92BF92CF9276
:1052F000DF92EF92FF920F931F93CF93DF93462E8F
:105300004A015901662309F4C4C09C01E90100E087
:10531000FF241FEFDD2466247724B2E05B2E3324C4
:105320003394CE010E940029F301E355F94F8083A5
:10533000C0802FE0C222C39440E050E012C01E257E
:105340001F7BF1F4F501E00FF11D3082FF2009F021
:1053500070C0DD24D3940F5F4F5F5F4F1E2D4C153F
:1053600088F5642FFE01E40FF51FE0802E2D30E05C
:10537000C9018F7090700F9709F455C0DD20F9F6C0
:10538000F501E00FF11D5082EF2DF0E0D401AE0FDA
:10539000BF1FEC926295607FE95DF94F6083F394E3
:1053A0000024220F331F001C220F331F001C232F49
:1053B000302DDD24D394D2220F5F4F5F5F4F1E2D1F
:1053C0004C1578F20894611C711C6096641408F402
:1053D000A8CF003408F061C08F2DF501E00FF11D5A
:1053E00010820F5F0034C8F39FE39F1550F09FEFCA
:1053F000EF2DF0E0E95DF94F9083F3942FE32F1543
:10540000B8F7DF91CF911F910F91FF90EF90DF9050
:10541000CF90BF90AF909F908F907F906F905F9054
:105420004F903F900895F501E00FF11D1082DD24AB
:1054300092CFEF2DF0E03197E80DF91DE082FA945C
:10544000EF2DF0E0F394E95DF94FA081AF70BA2F32
:10545000BF5F808182958F70682F70E0CB018B0FCA
:10546000911D40970CF0BA2F0024220F331F001C0F
:10547000220F331F001C232F302DDD24D394D22282
:1054800062957295707F7627607F7627B62BB08302
:1054900062CF00E0FF2480E0A0CF8F2DA5CF2F9218
:1054A0003F924F925F926F927F928F929F92AF92B4
:1054B000BF92CF92DF92EF92FF920F931F93CF9301
:1054C000DF935C01562E3A016901662309F45DC041
:1054D000482EEC0130E060E0EE24FF24FA9480E0F6
:1054E00000E010E05FE04EE0342E2DE0222E9DEA39
:1054F000892E96E0992E800E911EF40170817F70A6
:105500007F5FDE0190E0442D41950BC05C9322301B
:1055100089F0E42EEA0E3F5F9F5F1196822F971766
:10552000D0F4F601E30FF11D2081213079F78823B3
:1055300049F45C93F301E60FF11DF0806F5FFC927C
:1055400022E0E7CF5C93F501EE0DF11D80818064D0
:105550008083FC92DECF903158F4FE01E90FF11DFB
:1055600030829F5F05C0FE01E90FF11D50839F5FF0
:105570009031C8F3F401808184FD2F860F5F1F4FA7
:105580006096822F051508F4B2CFDF91CF911F915D
:105590000F91FF90EF90DF90CF90BF90AF909F90D2
:1055A0008F907F906F905F904F903F902F900895D5
:1055B00080919A050E940D13882339F08091DD05B2
:1055C0008093A90681E080932206089510928905B0
:1055D00084E20E948B1510925F0480E00E948B157C
:1055E0000E948E170E9492160E9417168091D7046F
:1055F0000E94251680E00E94D61C089581E08093C9
:10560000890584E20E9453150E94171680E00E94CB
:10561000251680E00E94D61C0895109224060E9450
:1056200092160E9417160E948E178091D7040E942E
:1056300025161092200681E20E948B1580E00E94C0
:10564000D61C109210078CEF0E944D0F08951092F7
:10565000990581E08093200681E20E94531580E045
:105660000E94D61C80912E04882321F480912F045F
:1056700080FDFCCF10922F041092430410928404FA
:10568000809184048093860481E080932406809333
:1056900010078AEF0E944D0F0895809170048823AF
:1056A00011F480E0089581E00E943613882321F0F0
:1056B00081E080937104089581E00E94F7128823AD
:1056C00081F380E00E94E112882359F382E0809305
:1056D000710481E0089588E00E94E112882369F056
:1056E0009091A90688E080939A059093DD0583E068
:1056F0008093A90681E080932206089580912E046C
:10570000823011F080E008950E947C0F809305079D
:1057100080E00895AF92BF92CF92DF92EF92FF9216
:105720000F931F93CF93DF935B01C82EDD24C294A8
:10573000D29450EFD522DC24C522DC24EE24C0E034
:10574000D0E0FF24F39405C02196F394F1E1FF1615
:10575000B1F085010C0F1D1FC6018C0F9D1F0E940B
:10576000E11DF8018083EE2079F780818F708E3003
:1057700059F7EF2C2196F394F1E1FF1651F7EE2043
:10578000A1F490E1F50187858F708D30B9F0892FF4
:1057900081508F70DF91CF911F910F91FF90EF900B
:1057A000DF90CF90BF90AF9008959E2D915051F70C
:1057B00091E0F50187858F708D3049F7903110F0B9
:1057C0008EE1E8CF892F81508F708061E3CFBF9247
:1057D000CF92DF92EF92FF920F931F93CF93DF93BD
:1057E0006801E82EFF24EE0CFF1CE60EF11CEE0C07
:1057F000FF1CEE0CFF1CEE0CFF1CE40EF11CE294EF
:10580000F29470EFF722FE24E722FE2430E0229586
:105810003295307F3227207F3227B22E222379F033
:10582000C0E0D0E086010C0F1D1FC7018C0F9D1F2B
:105830000E94E11DF80180832196CB1598F3DF913A
:10584000CF911F910F91FF90EF90DF90CF90BF907D
:105850000895EF92FF920F931F93CF93DF93182F2A
:10586000062F0E945717E12EFF24EE0CFF1CEE0CB2
:10587000FF1CEE0CFF1CE00EF11CE294F294A0EF72
:10588000FA22FE24EA22FE24C0E0D0E0FE01EE541B
:10589000F94F8081BE016E0D7F1D0E949D1D2196D6
:1058A000C031D10599F70E945717DF91CF911F9111
:1058B0000F91FF90EF900895CF92DF92EF92FF92B9
:1058C0000F931F93CF93DF93E22E6801082F10E010
:1058D000000F111F060F111D000F111F000F111FC8
:1058E000000F111F040F111D02951295107F102734
:1058F000007F1027FF24E294F29480EFF822FE2428
:10590000E822FE24FE2C82E00E9453150E945717C5
:10591000EE2089F0C0E0D0E0F601EC0FFD1F8081A1
:10592000B8016C0F7D1F0E949D1D84E00E94420EF5
:105930002196CF1588F382E00E948B150E9457179D
:10594000DF91CF911F910F91FF90EF90DF90CF905B
:105950000895EF92FF920F931F93CF93DF93182F29
:10596000062F0E945717E12EFF24EE0CFF1CEE0CB1
:10597000FF1CEE0CFF1CE00EF11CE294F29440EFD1
:10598000F422FE24E422FE24C0E0D0E0CE018E0DFD
:105990009F1D0E94E11DFE01EE54F94F8083219668
:1059A000C031D10599F710925F0480E00E94A815DC
:1059B0000E945717DF91CF911F910F91FF90EF90A9
:1059C000089580912E04882349F40E94A5008091B7
:1059D0002E04813049F00E948C1208950E94B00379
:1059E00080912E048130B9F70E94931208959F92FE
:1059F000AF92BF92CF92DF92EF92FF920F931F93DD
:105A000081E08093A9068093220600E011E032E055
:105A1000F32E2FE0E22E94E0D92E86E0C82EB7E0D8
:105A2000BB2EAAE0AA2EF0E29F2E0E94A61480911F
:105A3000A906863009F46FC0873008F0AAC081300B
:105A400009F456C1843089F780912206882339F001
:105A500010922206109365041092630400E0809176
:105A60009A050E940D13882331F18091DD05809302
:105A7000A906109322060023E1F080916304882395
:105A800011F41093630480916304813210F09092BA
:105A900063049091000280916304981751F0809103
:105AA0006304809300026091000287E090E00E940E
:105AB0005002109238040E945414282F882381F039
:105AC000809163048A9DC0011124809363048091B6
:105AD00063048150820F80936304F092650401E0B7
:105AE00080916504882309F4A0CF909100028091F1
:105AF0006504823009F4FDC1892F90E00E94EB011A
:105B000010933804109265040E94A6148091A9068F
:105B1000863009F091CF80912206882339F01092C7
:105B20002206109265041092630400E080919A05A9
:105B30000E940D13882349F08091DD058093A9060A
:105B400010932206002309F0D7C1809163048823B3
:105B500009F475C120916304213009F453C12091E7
:105B60006304223009F422C180916504813009F474
:105B70003EC180916504823009F057CF10926504D0
:105B80000E941716809198040E9425160E945717AC
:105B90004CCF873009F450C08F3009F046CF809148
:105BA0002206882349F01092220610936504809102
:105BB000CE048093640400E080919A050E940D1346
:105BC000882349F08091DD058093A9061093220671
:105BD000002309F068C10E94DA13882369F0982F26
:105BE0009150933048F480919204981729F0909343
:105BF00092041093650401E080919204813009F4CD
:105C000036C180916504882309F40FCF1092650492
:105C10000E9400170E941716809192048F5F0E94C5
:105C2000A01680919204813009F0FFCE80919504F6
:105C300081500E942516F9CE80912206882321F0FA
:105C4000109222061093650480919A050E940D130C
:105C5000882351F08091DD058093A90610932206D8
:105C60008091650481FD31C10E94DA13882389F097
:105C7000982F9150933068F480912E04981749F032
:105C800090932E040E94E12C8091650483608093A0
:105C9000650483E00E94F712882379F080916804FC
:105CA0008F5F80936804809168048170809368049A
:105CB000809165048360809365048091650480FF12
:105CC000B4CE809165048E7F809365040E94001796
:105CD00080912E048F5F0E94A01683E20E948B1594
:105CE00080916804882309F414C10E9457179DCE3F
:105CF00080912206882331F0109222060E9402161B
:105D00000E94571787E10E943613882359F090911B
:105D1000A90687E180939A059093DD05B092A906C4
:105D20001093220688E00E943613882359F0909140
:105D3000A90688E080939A059093DD05C092A90694
:105D40001093220681E00E943613882351F080913F
:105D5000A90610939A058093DD05D092A9061093A9
:105D600022068EE00E943613882359F09091A906EE
:105D70008EE080939A059093DD05E092A90610933A
:105D800022069091CD048091D304891709F44DCE59
:105D90008091CD048093D3041F910F91FF90EF90D9
:105DA000DF90CF90BF90AF909F9008959091CE04D8
:105DB00080916404981759F08091CE048093640414
:105DC00020936504809164048093980401E089E045
:105DD0000E940D13882309F4C7CE109263048BE14F
:105DE0000E948B1580916504813009F0C2CE10921B
:105DF00065040E9417168091AB040E9425160E942C
:105E0000571713CE9091CE0480916404981759F0DF
:105E10008091CE048093640420936504809164048F
:105E20008093AB0401E08AE00E940D13882309F4FB
:105E300096CE109263048CE10E948B1590CE8AE07E
:105E40000E94F712882309F068C089E00E94F712C7
:105E5000882309F47FCE8BE10E945315F0926304EE
:105E6000F09265048091CE048093640473CE909187
:105E700064048091CE04981709F4C3CE8091CE04B7
:105E800080936404909164049F5F923008F451C041
:105E900080919504981709F4B4CE909395041093CB
:105EA000650401E0AECE809195046091920490E08B
:105EB000019782959295907F9827807F9827682BED
:105EC0008AE090E00E94500286CE8091680490E0C3
:105ED0008170907082959295907F9827807F982707
:105EE00060912E046F70682B82E090E00E94500257
:105EF000BBCE9091630400CE83E090E06091AB0450
:105F00000E94500284E090E0609198040E94500248
:105F10001CCE83E20E945315E8CE8CE10E945315FB
:105F200010936304109365048091CE0480936404FD
:105F30008CCF92E0ADCF0F931F938091AA068093F0
:105F4000B106809126068823C9F08091DE058093F2
:105F5000C2068091960580930307809198058093EF
:105F60001F068091260680932506109226068091B2
:105F70006204823088F01F910F9108959091030779
:105F8000809196059817B9F380916204823098F752
:105F900080919605809303078091C2066091030764
:105FA00040911F062091250609E616E00E94E72B86
:105FB00060911F068091AB069091AC060E9420294B
:105FC0001F910F9108951092100780E00E94D61C37
:105FD0008CEF0E944D0F80912E04813011F00E94B1
:105FE0006212109267061092840480918404809358
:105FF00086041092970589E696E09093AC0680930C
:10600000AB068091D3048D3031F0833021F08B309A
:1060100011F0873011F40E949B2F80913C0488235B
:1060200061F480913B04882309F4089580913B0436
:106030000E94270F10923B04089580913C040E9417
:10604000270F10923C04EDCF1F93DF93CF930F9255
:10605000CDB7DEB780E00E94D61C10926706109282
:106060002F041092430410927204109284048091C1
:106070008404809386041092970589E696E09093B5
:10608000AC068093AB0610911F060E9400298983FD
:1060900089818F708F5F8093EB0310939C058981BA
:1060A00084FD1BC086E08093E90383E080931007A2
:1060B0008AEF0E944D0F80912E04813011F00E94D2
:1060C0009A1283E08093360410923B0410923C04B1
:1060D0000F90CF91DF911F91089588E0E4CFEF9268
:1060E0000F931F93982F882309F495C0813029F0CE
:1060F00080E01F910F91EF900895809122068823F0
:1061000009F0F9C00E94DA13882399F1982F915071
:1061100080912606882341F480911F06809398057C
:106120008091C2068093DE0580919805891770F4EE
:1061300080919805981B9F5F909326068091260674
:10614000853008F446C184E08093260680911007CC
:10615000882309F441C180911F0660912506409172
:1061600098052091260600919C05E09096050E94D6
:10617000461884E10E94F712882309F0DEC085E109
:106180000E94F712882309F0CEC08091100788235F
:1061900021F590910307809196059817F1F0809171
:1061A0009605809303078091C20660910307409192
:1061B0001F062091250609E616E00E94E72B809134
:1061C0001F066091250640919805209126060091B2
:1061D0009C05E09096050E94461880911007882340
:1061E00029F480912606882309F0D4C00E94F41374
:1061F000982F882309F47CCF8091630491509817DD
:1062000009F076CF8091DD058093A90681E0809327
:10621000220680E06ECF0E94DA13982F8823D1F5F2
:1062200084E10E94F712882309F49FC0109296051A
:1062300088E00E94531581E00E948B158091100721
:10624000882309F055CF9091030780919605981700
:1062500009F44ECF80919605809303078091C20682
:106260006091030740911F062091250609E616E07C
:106270000E94E72B80911F066091250640919805AA
:106280002091260600919C05E09096050E944618F4
:1062900080E02FCF8091D8048093DE0501E0009349
:1062A0002606192F11501093980584E10E94E112DF
:1062B000882309F44BC01092960588E00E9453157C
:1062C00081E00E948B15109363048091A90680934E
:1062D000DD058DE08093A90681E08093220610926F
:1062E000AA0680911007882309F44FC081E01F910E
:1062F0000F91EF9008951092220690937004809170
:106300001F06609125064091980520912606009170
:106310009C05E09096050E9446180E94DA13882397
:1063200009F427CFF3CE81E08093960588E00E94A0
:106330008B1581E00E94531528CF1092960588E0B6
:106340000E94531581E00E948B1519CF85E10E94B0
:10635000E112882309F4B7CF0093960588E00E94E4
:106360008B1581E00E945315AECF85E10E94F71294
:10637000882309F463CF81E08093960588E00E942A
:106380008B1581E00E94531559CF82E00E94EF28BF
:1063900081E0ADCF8091DE058093C20680919605A5
:1063A000809303078091980580931F0680912606AD
:1063B00080932506109226068091C20660910307FD
:1063C00040911F062091250609E616E00E94E72B62
:1063D0000DCF80912606B8CE8091DE058093C2064F
:1063E00080919605809303078091980580931F06FE
:1063F0008091260680932506109226068091C2067B
:106400006091030740911F062091250609E616E0DA
:106410000E94E72BA0CE2F923F924F925F926F92F5
:106420007F928F929F92AF92BF92CF92DF92EF9224
:10643000FF920F931F93DF93CF930F92CDB7DEB7E9
:106440000E94A6141092AA068091AA068093B10613
:1064500080911007882311F40C949F3B84E0809373
:10646000A90681E080932206662499248824552475
:106470007724739438E0432E26E0322E93E0292EC1
:106480000E94A6141091A9061830D9F0193008F00E
:106490004CC0153009F49EC4163008F096C0113077
:1064A00009F431C2143009F40CC40E947E2B8823F5
:1064B00039F70E944D2B0E94A6141091A90618309E
:1064C00029F780912206882349F0109222060E9423
:1064D000021683E20E9453157092620480919A051D
:1064E0000E940D138823A1F08091DD058093A906F9
:1064F00070922206109262048091C2066091030796
:1065000040911F062091250609E616E00E94E72B20
:106510000E94DA13882309F00FC50E94F413882320
:1065200021F281500E943E18C0CF1B3009F4DEC218
:106530001C30D0F5193009F485C21A3009F0B5CFF6
:10654000809122068823F9F01092220680E00E94B2
:1065500053150E9457178091C2066091030740911E
:106560001F062091250609E616E00E945C2C80E0BB
:106570000E948B150E94571784E08093A9067092A1
:1065800022061092620480916504882339F084E029
:106590008093A9067092220610926504809165048A
:1065A0008F5F8093650481CF1C3009F47CC11D305E
:1065B00009F07BCF81E00E946F308091A9068D3079
:1065C00009F473CF1092700470CF163009F4FCC038
:1065D000173009F06ACF80912206882389F1109242
:1065E00022060E9402166091250689E696E043EC99
:1065F00056E02DE935E00E946E2980E00E94531597
:106600001092650489E08093630410926404809181
:106610002506882391F020E0E22FF0E0E355F94FC2
:106620009081809164048F5F9F70890F80936404D0
:106630002F5F80912506281778F366249924552426
:1066400080E00E943613882311F06624639488E06A
:106650000E943613882311F012E0612E87E10E9418
:106660003613882311F0B3E06B2E809163048930D8
:1066700009F4E7C680916304813009F4BCC68091B7
:106680006304882309F491C580916304882329F069
:1066900080916304807F09F45FC0109163048EE0F1
:1066A0000E94F712882351F08091630480618093E7
:1066B000630485E080936504F2E05F2E8FE00E9422
:1066C000F712882351F08091630480628093630401
:1066D00085E0809365045524539484E10E94F71269
:1066E000882349F08091630480648093630485E08B
:1066F0008093650455248EE00E940D13882341F099
:1067000080916304807E8093630484E080936504B9
:106710008FE00E940D13882341F080916304807DF7
:106720008093630484E08093650484E10E940D13E8
:10673000882341F080916304807B8093630484E02C
:106740008093650480916504853009F44EC580917D
:106750006504843009F460C580916304883009F4CD
:106760003CC48091650490E083709070892B09F09F
:106770004CC4662009F499CE6091250689E696E01E
:1067800043EC56E02DE935E00E944F2A8091C20685
:106790006091030740911F062091250609E616E047
:1067A0000E945C2C91E0691609F446C5E2E06E1681
:1067B00009F474C0F3E06F1609F077CE87E0809398
:1067C000A9067092220671CE809122068823D9F004
:1067D000109222060E9402166091250689E696E034
:1067E00043EC56E02DE935E00E946E2984E20E94D8
:1067F00053151092650410926404E3E6E093630479
:1068000066249924882480E00E943613882311F09E
:106810006624639488E00E943613882311F082E096
:10682000682E80916304833609F41EC58091630449
:10683000813009F428C580916304833009F486C54A
:1068400080916304882309F451C48091650490E029
:1068500083709070892B09F019C4662009F425CE45
:106860006091250689E696E043EC56E02DE935E097
:106870000E944F2A8091C2066091030740911F0633
:106880002091250609E616E00E945C2C91E069162D
:1068900009F4D2C4E2E06E1609F007CE3092A906E0
:1068A0007092220602CE80912206882389F01092EF
:1068B00022069091600480912506981709F42CC651
:1068C000709265048091DD058093A906709222067E
:1068D00080919A050E940D13882309F4E6CD8091DA
:1068E000DD058093A90670922206809165048823B5
:1068F00009F4B7C58DE00E948B1582E00E948B15CC
:106900000E945717D2CD809122068823E9F0109279
:10691000220680E00E9427020E94021682E20E9464
:1069200053151093700481E20E948B1580911F060D
:1069300060912506409198052091260600911F063A
:10694000E09096050E94461880E00E946F3080E03B
:106950000E94F712882329F085E08093A90670929F
:10696000220683E00E94F712882351F08091A90645
:1069700020929A058093DD054092A9067092220626
:1069800088E00E943613882321F03092A906709285
:10699000220687E10E943613882329F087E080933E
:1069A000A906709222068BE00E943613882359F0C4
:1069B0009091A9068BE080939A059093DD058093D2
:1069C000A906709222068DE00E943613882361F09A
:1069D0009091A9068DE080939A059093DD059CE047
:1069E0009093A906709222068091A906813011F039
:1069F0001092700480911007882329F084E080931E
:106A0000A906709222069091CD048091D304891733
:106A100009F44BCD8091CD048093D3040F90CF9196
:106A2000DF911F910F91FF90EF90DF90CF90BF907B
:106A3000AF909F908F907F906F905F904F903F901E
:106A40002F90089580912206882371F010922206DB
:106A500082E20E948B1581E00E94D61C80E00E9499
:106A6000D61C80E00E9427029091630480919B05D0
:106A70009817C9F09090630480919B0580936304FC
:106A800080916504833009F4AAC580916504823041
:106A900050F080919505882331F4E0916304F0E093
:106AA000E356FA4F708286E10E94F712882329F09C
:106AB00080919505882309F450C580916504833041
:106AC00009F4BFC386E10E940D13882309F4EDCCBD
:106AD00080916504823009F0E8CC7092650480E012
:106AE0000E94D61C82E00E948B15DFCC809122068A
:106AF000882361F01092220682E20E948B158FE0BB
:106B00000E9453150E9457171092650480919A05B0
:106B10000E940D13882309F442C08091DD05809303
:106B2000A9067092220680916504882391F58091D0
:106B3000C2063091030720911F0690E0880F991F2D
:106B4000830F911D880F991F880F991F880F991F18
:106B5000280F209361048091250680936004882388
:106B6000C1F090E0A0E0B0E0282F30E0229532950F
:106B7000307F3227207F3227FD01E759F94F80818E
:106B8000A152BA4F8C939F5FA92FB0E0A217B30711
:106B90009CF38FE00E948B158DE00E948B158DE099
:106BA0000E94F712882309F480CC80916504882321
:106BB00009F07BCC80916004882309F476CC709234
:106BC00065048091C2062091030710911F0690E092
:106BD000880F991F820F911D880F991F880F991F89
:106BE000880F991F180F80916104181709F45DCC64
:106BF0008DE00E94531582E00E9453150E945717A2
:106C00006091610480912506882309F440C0C62E56
:106C1000DD24C294D294A0EFDA22DC24CA22DC2440
:106C2000A12EBB24A294B294F0EFBF22BA24AF22CB
:106C3000BA24750100E010E0C6010E94E11D882E13
:106C40000759194FF8018083C7010E94E11DB60161
:106C50000E949D1D882DB7010E949D1D84E00E9409
:106C6000420E0894C11CD11C0894E11CF11C8E2D0D
:106C70008A19082F10E08091250690E08295929560
:106C8000907F9827807F982708171907ACF21091FA
:106C90001F0689E696E00E940029898389818F700A
:106CA0008F5F8093EB0310939C05898184FD51C510
:106CB00086E08093E90382E00E948B150E945717BB
:106CC000F4CB809122068823E9F0109222060E94DC
:106CD000021682E20E9453157092700481E20E94B3
:106CE000531580911F0660912506409198052091CB
:106CF000260600911F06E09096050E94461881E046
:106D00000E94270283E00E943613882309F445C0BD
:106D100080912606882309F00DC490910307809185
:106D20009605981781F080919605809303078091CE
:106D3000C2066091030740911F062091250609E6CF
:106D400016E00E94E72B6091250689E696E043EC69
:106D500056E02DE935E00E946E2980E090E0FC01CC
:106D6000E356FA4F1082019680349105C1F782E014
:106D700080936204109206071092640410926304D8
:106D800010926504109295057092670489E08093D3
:106D9000A9067092220699249A948091A9068430BB
:106DA00011F01092700480911007882321F47092E2
:106DB000A9067092220680916F04813009F075CB8C
:106DC00010926F049091CD048091D304891709F03B
:106DD00021CE6BCB809122068823C9F01092220627
:106DE0000E9402167092650489E696E00E940029CE
:106DF000282F2F702F5F2093630490E09295829547
:106E00008F7089279F7089278170809364048EE03A
:106E10000E947514823009F4D3C08AE00E94751470
:106E2000823009F4C4C089E00E947514823009F4EC
:106E3000B2C08FE00E94F712882399F02092650477
:106E400080916404882319F49CE0909363048091FA
:106E500064048F5F809364048091640481708093E4
:106E600064048091650480FF21C080916504815095
:106E70008093650480916404882309F4AAC18091F9
:106E80006304803108F4A8C381E08093630483E045
:106E90000E94531580916304882309F097C181E013
:106EA00080936304809163040E94301680E00E9406
:106EB0000D13882309F4F9CA809165048230B8F172
:106EC00082E08093620489E696E061E043EC56E05C
:106ED0002DE935E00E946E2990916304809164044D
:106EE000811180E191509F70892B8093AD0689E6D6
:106EF00096E061E043EC56E02DE935E00E944F2A30
:106F00008091C2066091030740911F0621E009E6C7
:106F100016E00E945C2C8091C206609103074091AC
:106F20001F06209125060E94E72B109262047092A2
:106F3000A90670922206B9CA182F1150812F0E94FB
:106F400036188091C20690910307E82EFF24EE0CBC
:106F5000FF1CE90EF11CEE0CFF1CEE0CFF1CEE0CEE
:106F6000FF1CE10EF11CE294F29450EFF522FE2496
:106F7000E522FE248701005F1F4F8FE0B7010E94CA
:106F80009D1D84E00E94420E0894E11CF11CE01655
:106F9000F10699F7C2CA8091630490E00E968F7053
:106FA00090708F5F809363042092650442CF80913C
:106FB00063048F708F5F809363042092650433CFE6
:106FC00080916504823008F482C3809163048F5FEE
:106FD000809363042092650420CFE92DF0E0E3560E
:106FE000FA4F5082939480916404981610F06624AE
:106FF000639470926504109263048091650490E03C
:1070000083709070892B09F4B4CB0E94171680917D
:1070100025068823B1F090E080E001C08E2FE92F93
:10702000F0E0E355F94FE081EF70EF5FE80F98165D
:1070300018F09E1608F4DCC29F5F80912506981711
:1070400068F384E00E948B1583E00E948B1588E032
:107050000E948B158091650480FD13C0F2E05F16DD
:1070600009F479C381E0581609F479C3552031F049
:1070700084E00E94531583E00E94531588E00E942B
:1070800053150E9457171092650473CB0E94171670
:10709000E92DF0E0E95DF94F80818F3FD1F010815B
:1070A00012951F7000810F70010F0F5F101738F0DD
:1070B00010C0812F0E944E161F5F101750F4809150
:1070C000650480FDF6CF812F0E9425161F5F1017E3
:1070D000B0F38091650480FFBFC1882D60E00E94FD
:1070E000A118109265040E945717B7CB86E10E9441
:1070F000F712882309F0B8C20E948C13882309F084
:1071000081C287E10E940D13882329F08FE3980E36
:107110009822709265048EE00E94F712882321F075
:1071200090E1892A709265048FE00E94F71288230B
:1071300021F0E0E28E2A7092650484E10E94F71249
:10714000882321F0F0E88F2A7092650485E10E947F
:10715000F712882321F080E4882A709265048EE07B
:107160000E940D13882321F09FEE892270926504FE
:107170008FE00E940D13882321F0EFED8E22709294
:10718000650484E10E940D13882321F0FFE78F221C
:107190007092650485E10E940D13882309F455CB94
:1071A0008FEB88227092650450CB86E10E943613E3
:1071B000882309F469CAE92DF0E0E356FA4F5080BC
:1071C0007092630482E0809365045ECA80916304D8
:1071D00067CE80916304813108F4FBC181E0809324
:1071E000630483E00E948B1555CE112309F0E8C19A
:1071F00080916304882309F4E3C1662029F4E92D12
:10720000F0E0E356FA4F508282E08093650480916B
:107210006504843009F0A0CA112359F080916304F9
:10722000882339F4939480916404981610F06624AE
:1072300063947092650490CA6092A90660922206D7
:1072400034C90E942414882309F43CCC82E0809342
:10725000650486E10E94E112882309F033CC709224
:1072600065040E94D61C2ECC88E00E940D13882352
:1072700009F4DCCA1092630470926504809163047F
:10728000813009F0D8CA86E10E940D13882309F0E5
:1072900023C28EE00E94F712882349F0882D809542
:1072A0008071FFEE8F22882A82E0809365048FE050
:1072B0000E94F712882349F0882D809580729FEDF7
:1072C0008922882A82E08093650484E10E94F71273
:1072D000882349F0882D80958078EFE78E22882AD0
:1072E00082E08093650485E10E94F712882349F0CB
:1072F000882D80958074FFEB8F22882A82E080930E
:1073000065040E948C13182F882309F494CA80E026
:107310000E94D61C85E00E94420E11501F7080EF23
:107320008822812AE82DF0E0EF73F070E451FC4FE1
:10733000482D4078808160E00E94BF1C82E08093ED
:10734000650480916304833009F07ACA0E948C132B
:10735000182F0E94A613882319F4112309F470CA68
:10736000E92DF0E0ED53F94F808280E00E94D61CB9
:1073700085E00E94420E93949FE3991518F41092B1
:10738000640499247092650410926304112309F433
:1073900057CA812E8A94EFE08E228EE00E94E1127D
:1073A000882311F0F0E18F2A8FE00E94E1128823F8
:1073B00011F080E2882A84E10E94E112882311F012
:1073C00090E8892A85E10E94E112882311F0E0E427
:1073D0008E2AE82DF0E0EF73F070E451FC4F482D59
:1073E0004078808160E00E94BF1C82E08093650449
:1073F0002092630425CA86E10E940D13882311F0B0
:10740000409263048EE00E94F712882329F082E004
:1074100080936504A2E05A2E8FE00E94F712882321
:1074200029F082E0809365045524539484E10E94FE
:10743000F712882309F423C982E080936504552458
:107440001EC987E10E940D13882309F413C9109205
:107450006304709265040EC9882D61E00E94A11832
:1074600040CE82E00E9453150E9457179091C206A9
:107470002091030730911F06809160048823B9F1A1
:10748000E92EFF24EE0CFF1CE20EF11CEE0CFF1C9B
:10749000EE0CFF1CEE0CFF1CE30EF11CE294F294C8
:1074A00050EFF522FE24E522FE248701A0E0B0E0A3
:1074B000FD01E152FA4F8081A759B94F8C93B80171
:1074C0000E949D1D84E00E94420E0F5F1F4F802F7F
:1074D0008E19A82FB0E08091600490E0829592957B
:1074E000907F9827807F9827A817B9070CF31091F1
:1074F0001F0689E696E00E940029898389818F70A2
:107500008F5F8093EB0310939C05898184FDE2C01B
:1075100086E08093E903EEC9992309F4D1C982E298
:107520000E948B158DE00E9453150E9457171092F0
:107530006504CEC98091DE058093C20680919605D0
:10754000809303078091980580931F0680912606FB
:107550008093250610922606EACB82E0809365048C
:107560000E940E14882311F020926504E0916304B8
:10757000F0E0E356FA4F82E08083E0916404F0E0AB
:10758000ED53F94F808080922306E82DF0E0EF73F1
:10759000F070E451FC4F482D4078808160E00E94FB
:1075A000BF1C80916304981639F090906304809119
:1075B00064048F5F8093640482E00E9453157DCA47
:1075C000939480916404981608F417CE662463940B
:1075D0001BCE8091630403CE8091630456CC0E943D
:1075E0000E14882309F051CA82E0809365044DCAC5
:1075F000992D981B8091650480FF9DC0892F0E9462
:107600004E161FCD882E8A94FFE08F228EE00E94B6
:10761000E112882311F080E1882A8FE00E94E112B4
:10762000882311F090E2892A84E10E94E1128823E4
:1076300011F0E0E88E2A85E10E94E112882311F022
:10764000F0E48F2AE82DF0E0EF73F070E451FC4F86
:10765000482D4078808160E00E94BF1C82E08093CA
:107660006504209263044DCDE92DF0E0ED53F94F10
:1076700080808EE00E94E112882311F0F0E18F2AD1
:107680008FE00E94E112882311F080E2882A84E1D1
:107690000E94E112882311F090E8892A85E10E9476
:1076A000E112882311F0E0E48E2AE82DF0E0EF7378
:1076B000F070E451FC4F482D4078808160E00E94DA
:1076C000BF1C82E0809365047092630415CD109214
:1076D00063047BCC88E01DCFE92DF0E0ED53F94F3A
:1076E00080828EE00E94E112882381F588248FE059
:1076F0000E94E112882311F0F0E28F2A84E10E94B7
:10770000E112882311F080E8882A85E10E94E112C5
:10771000882311F090E4892A80E00E94D61C93947B
:10772000EFE3E91518F4109264049924709265044B
:1077300010926304AECD892F0E94251682CC81E081
:107740008093A906809322060C94343200E1802EA7
:10775000CECF88E0AECA84E00E94531592CC83E07D
:107760000E9453158ECC0F931F93CF93DF93EC01A0
:10777000442319F18B0150E070E020E030E0F90182
:10778000E355F94F60816F706F5FD80190E0FE01A3
:10779000E50FF11D80818D939F5F5F5F9617B8F3B2
:1077A000760F2F5F3F4F005F1F4F241740F3872F47
:1077B000DF91CF911F910F91089570E0872FDF9196
:1077C000CF911F910F910895BF92CF92DF92EF92C8
:1077D000FF920F931F93CF93DF936B01B42E44233B
:1077E00069F17C0110E000E0C0E0D0E0C7010E9438
:1077F0000029FE01E355F94F808320812F702F5F10
:10780000D70190E08D91F601E10FF11D80839F5F1C
:107810001F5F9217B8F3020F219680E190E0E80E07
:10782000F91ECB1518F3802FDF91CF911F910F9187
:10783000FF90EF90DF90CF90BF90089500E0F3CFDE
:10784000CF92DF92EF92FF920F931F93DF93CF932C
:10785000CDB7DEB7C054D0400FB6F894DEBF0FBE30
:10786000CDBF109265041092630482E0809362049D
:107870004091250689E696E06E010894C11CD11C52
:10788000B6010E94E43BE82E809164048E1510F04E
:1078900010926404809125068823C1F090E030E0C6
:1078A000E32FF0E0E355F94F20812F702F5F80E048
:1078B000E92FF0E0E95DF94F80838F5F9F5F8217CA
:1078C000B8F33F5F80912506381750F30E94A61445
:1078D00080911007882309F4C5C184E00E946029C3
:1078E000FF240E94A6141091A906113071F01430E3
:1078F000E1F10E947E2B8823A1F70E944D2B0E946C
:10790000A6141091A906113091F70E9466298823C8
:1079100009F0F4C086E10E943613882329F0809193
:107920006604882309F088C18091A906813011F08E
:107930001092700480911007882309F070C10E9492
:10794000AB288823B1F210926204C05CDF4F0FB6FF
:10795000F894DEBF0FBECDBFCF91DF911F910F9185
:10796000FF90EF90DF90CF9008950E9466298823C2
:1079700009F037C110E086E10E943613882309F030
:10798000D0C087E10E943613882309F0E6C086E163
:107990000E940D13882309F0FCC087E10E940D139B
:1079A000882309F001C186E10E94F712882309F0BB
:1079B00006C18EE00E94F712882339F08F2D809542
:1079C00080719FEEF922F82A12E08FE00E94F712F0
:1079D000882339F08F2D809580729FEDF922F82A47
:1079E00012E084E10E94F712882339F08F2D8095F0
:1079F00080789FE7F922F82A12E085E10E94F712C9
:107A0000882339F08F2D809580749FEBF922F82A16
:107A100012E00E948C13282F882361F08F2D90E0B4
:107A20008F7090700D9734F421502F7080EFF822F2
:107A3000F22A12E088E00E94F712882309F44AC073
:107A40008F2D90E08F7090700D970CF4ECC090EF3C
:107A5000F92200E010E080916404F601E80FF11DC6
:107A6000F08240912506C60169E676E00E94B33BAC
:107A7000E82E81E0809366040D301105BCF58F2D52
:107A800061E00E94A11884E20E9453150E9417161B
:107A9000E0916404F0E0E95DF94F80810E942516D1
:107AA0000E9457178091A906843011F0109270043B
:107AB00080911007882309F4AEC080916F04813053
:107AC00009F017CF10926F040E94AB28882309F4A5
:107AD00010CF39CF123009F4C9C0113019F70F2D6A
:107AE00010E00F7010700D3011054CF28F2D60E01A
:107AF0000E94A11884E20E948B15C8CF0E94021632
:107B000082E20E9453151093700481E20E948B154B
:107B100080916604882309F4A1C082E00E946F1559
:107B2000F9CE809164048F5F809364048091640433
:107B30006E2D0E94D7459093640480916404F601F1
:107B4000E80FF11DF08082E00E94531511E087E1FB
:107B50000E943613882309F41ACF809164046E2D95
:107B600070E090E00197860F971F0E94F745809381
:107B7000640480916404F601E80FF11DF08080E058
:107B80000E94531511E086E10E940D13882309F429
:107B900004CF82E00E948B150E94571787E10E9454
:107BA0000D13882309F4FFCE80E00E948B150E94FC
:107BB000571786E10E94F712882309F4FACE80E075
:107BC0000E94E112882309F4F4CE80919B058093F2
:107BD000640480916404F601E80FF11DF08011E067
:107BE000E8CE0E94021682E20E94531581E0809343
:107BF000700481E20E945315809166048823C1F0CD
:107C000082E00E946F1580916404F601E80FF11D77
:107C1000F08011E0B0CE81E00E9460294ECF84E078
:107C20000E9460298CCE8FE0F82E0FE010E013CF79
:107C300082E00E948B15E7CF82E00E948B15809135
:107C4000C2066091030740911F062091250609E6B0
:107C500016E00E945C2C1092660466CE82E00E94C0
:107C60008B1558CE81E00E9460293ACE0F2D10E08E
:107C70000F701070F0CE3F924F925F926F927F9292
:107C80008F929F92AF92BF92CF92DF92EF92FF922C
:107C90000F931F93DF93CF93CDB7DEB7C058D0407B
:107CA0000FB6F894DEBF0FBECDBF109265041092E0
:107CB000630482E08093620440912506B1E4CB2EF8
:107CC000D12CCC0EDD1E89E696E0B6010E94E43B85
:107CD000E82E0E94A61480911007882309F42CC670
:107CE00084E00E9460299924442488245524AA24ED
:107CF000AA94BB24332433943E010894611C711C64
:107D00000E94A6141091A9061F30A9F0103108F0A6
:107D100088C0113009F4B8C2143009F44CC20E9472
:107D20007E2B882369F70E944D2B0E94A614109188
:107D3000A9061F3059F70E946629882309F09BC4C1
:107D40000E94D82A86E10E94F712882309F08AC48B
:107D500089E00E94F712882309F0D5C28AE00E94C8
:107D6000F712882309F0C7C286E10E940D13882309
:107D700009F0BDC289E00E940D13882309F0B3C247
:107D80008AE00E940D13882309F0A9C28DE00E94A9
:107D9000F712882329F080916004882309F031C507
:107DA00091E0991609F4DBC3A2E09A1609F4D3C353
:107DB000B3E09B1609F0B3CF30926604682D70E0F3
:107DC000842D992787FD9095860F971F850D911D0E
:107DD0000E94F745582EEE2099F020E030E0F601A1
:107DE000E20FF31F852D820F682D0E94D745D30126
:107DF000A90FB11D8C9180832F5F3F4F2E1578F313
:107E000040912506C60169E676E00E94B33B4091A9
:107E1000250689E696E0B6010E94E43BE82E992407
:107E20007ECF113109F41BC1113108F480C0123129
:107E300009F075CF0E946629882309F056C40E9474
:107E4000D82A8CE00E94F712882309F077C38CE0CF
:107E50000E940D13882309F06DC38EE00E94F71273
:107E6000882309F05DC38FE00E94F712882309F090
:107E70004DC384E10E94F712882309F03DC385E1D8
:107E80000E94F712882309F02DC388E00E94F712A0
:107E9000882309F01DC38EE00E940D13882309F08A
:107EA000EFC28FE00E940D13882309F0F2C284E133
:107EB0000E940D13882309F0F5C285E10E940D137D
:107EC000882309F0F8C288E00E940D13882309F086
:107ED000FBC2992009F423CF30926604EE2009F406
:107EE0008FCF860110C00E97F9F08F2D8A21D8010F
:107EF0009C919B21892BF80181938F018E2F8C19E6
:107F00008E1508F07DCF0E94E000F82E90E08F7073
:107F100090708D30910539F7E7EFFE228F2D90E0BC
:107F20008F7090700E9709F7F7EFFF22DECF0E9457
:107F30006629882309F09EC20E94D82A8CE00E94FC
:107F4000F712882309F0E7C187E10E94F71288231E
:107F500009F0ECC180E00E94F712882309F0F1C11A
:107F60008CE00E940D13882309F0F6C187E10E947E
:107F70000D13882309F0F9C180E00E940D138823B6
:107F800009F0FCC18EE00E94F712882309F0FFC1BE
:107F90008FE00E94F712882309F008C284E10E9452
:107FA000F712882309F011C285E10E94F712882395
:107FB00009F01AC288E00E94F712882309F023C250
:107FC0008EE00E940D13882309F02CC28FE00E94DE
:107FD0000D13882309F02FC284E10E940D1388231A
:107FE00009F032C285E10E940D13882309F035C2E1
:107FF00088E00E940D13882309F038C2992009F403
:108000008ECE30926604E2E09E1609F4D0C3F4E00E
:108010009F1609F446C4B1E09B1609F003C4EE2094
:1080200009F4EECE860107C00F5F1F4F802F8C1919
:108030008E1508F0E5CE0E94E000F82EEFE1E8177B
:1080400098F30E94E000D8012C916E2D0E94D74534
:10805000F601E90FF11D80818C932083E5CF0E940A
:108060006629882309F0F9C20E94D82A8CE00E9470
:10807000F712882309F0E8C28CE00E940D138823D0
:1080800009F0DEC28EE00E94F712882309F0CEC20A
:108090008FE00E94F712882309F0BEC284E10E949B
:1080A000F712882309F0AEC285E10E94F7128823F7
:1080B00009F09EC288E00E94F712882309F08EC260
:1080C0008EE00E940D13882309F084C28FE00E9485
:1080D0000D13882309F05FC284E10E940D138823E9
:1080E00009F062C285E10E940D13882309F065C280
:1080F00088E00E940D13882309F068C28DE00E9479
:10810000F712882329F080916004882309F043C086
:10811000192D10FF04CE3092660411FDEFC2EE203F
:1081200041F1860106C00F5F1F4F802F8C198E15FD
:1081300000F50E94E000F82EBFE3B817A0F30E94FC
:10814000E000F82E90E08F7090708D30910509F46A
:1081500004C30E9709F4FEC29F2D9A21D8018C9179
:108160008B21982B9C930F5F1F4F802F8C198E159E
:1081700000F3BEEF9B2240912506C60169E676E03A
:108180000E94B33B4091250689E696E0B6010E9425
:10819000E43BE82EC4CD892D80958270B1E09B220E
:1081A000982A8DE00E948B15192D91FCA2C388247A
:1081B0000E945717AECF0E946629882309F07FC21C
:1081C00084E00E943613882309F072C285E00E9481
:1081D0003613882309F065C282E10E943613882392
:1081E00009F058C281E10E943613882309F04BC27E
:1081F00086E10E943613882329F080916604882343
:1082000009F0EDC287E10E943613882329F080919E
:108210006604882309F0B2C28091A906843041F037
:108220001092700482E00E948B1582E20E948B15EE
:1082300080911007882309F48AC180916F048130EE
:1082400009F06DCD10926F040E94AB28882309F4C9
:1082500066CD10926204C058DF4F0FB6F894DEBFAF
:108260000FBECDBFCF91DF911F910F91FF90EF9087
:10827000DF90CF90BF90AF909F908F907F906F9046
:108280005F904F903F9008950E946629882389F45B
:108290008091A906813011F010927004809110072E
:1082A000882309F027C20E94AB28882309F437CD20
:1082B000D0CF0E94021682E20E94531510937004E0
:1082C00081E20E948B1580916604882309F4A6C27E
:1082D00082E00E946F1581E00E942702D9CF8CE1D5
:1082E0000E948B1553CD8BE10E948B1549CD82E006
:1082F0000E948B153FCD8CE10E9453159F2C9394C7
:108300004424439431CD8BE10E9453159F2C9394C8
:1083100044244A9423CD8EE00E94531599249394CB
:1083200087E10E94F712882309F414CE80E00E94AE
:108330005315F2E09F2E80E00E94F712882309F483
:108340000FCE82E20E945315E3E09E2E8CE00E9445
:108350000D13882309F40ACE8EE00E948B1587E165
:108360000E940D13882309F407CE80E00E948B152C
:1083700080E00E940D13882309F404CE82E20E945B
:108380008B158EE00E94F712882309F401CE84E059
:108390000E94531574E0972E60E1A62E5FEEB52E75
:1083A0008FE00E94F712882309F4F8CD83E00E9441
:1083B000531544E0942E30E2A32E2FEDB22E84E12B
:1083C0000E94F712882309F4EFCD88E00E9453152C
:1083D00094E0992E80E8A82E0FE7B02E85E10E9448
:1083E000F712882309F4E6CD81E00E94531514E0CA
:1083F000912EB0E4AB2EAFEBBA2E88E00E94F712BC
:10840000882309F4DDCD84E20E945315F4E09F2E09
:10841000EFE0AE2E70EFB72E8EE00E940D13882392
:1084200009F4D4CD84E00E948B158FE00E940D13D7
:10843000882309F4D1CD83E00E948B1584E10E944A
:108440000D13882309F4CECD88E00E948B1585E1B9
:108450000E940D13882309F4CBCD81E00E948B1577
:1084600088E00E940D13882309F4C8CD84E20E949D
:108470008B15C4CD89E10E945315992444245CCD09
:1084800084E00E948B158FE00E940D13882309F46D
:108490000ECD83E00E948B1584E10E940D1388238A
:1084A00009F40BCD88E00E948B1585E10E940D1325
:1084B000882309F408CD81E00E948B1588E00E9492
:1084C0000D13882309F405CD84E20E948B1501CD9C
:1084D00084E20E945315992493942FE0A22E90EFEA
:1084E000B92ED9CC81E00E9453159924939440E48D
:1084F000A42E3FEBB32EC9CC88E00E9453159924DB
:10850000939460E8A62E5FE7B52EB9CC83E00E9475
:10851000531599249394E0E2AE2E7FEDB72EA9CCAB
:1085200084E00E94531599249394A0E1AA2EFFEEB3
:10853000BF2E99CC8EE00E948B158FCC8EE00E94CE
:10854000531599249394AA24AA94BB2480CC81E047
:108550000E94602972CE442009F02ECCE0CB44204A
:1085600009F4DDCB90926604EE2089F0342D3E0DA7
:10857000D60120E0822F830F6E2D0E94D745F30194
:10858000E90FF11D8D9180832F5F2E1598F3409197
:108590002506C30138CC83E00E948B1584E10E943C
:1085A0000D13882309F49ECD88E00E948B1585E188
:1085B0000E940D13882309F49BCD81E00E948B1546
:1085C00088E00E940D13882309F498CD84E20E946C
:1085D0008B1594CD84E00E948B1578CD84E20E94A7
:1085E0005315A1E09A2A1FE0A12EB0EFBB2E68CD53
:1085F00081E00E94531591E0992A80E4A82E0FEBA8
:10860000B02E58CD88E00E94531581E0982A20E8CA
:10861000A22E9FE7B92E48CD83E00E945315F1E0CA
:108620009F2A40E2A42E3FEDB32E38CD84E00E9475
:108630005315E1E09E2A60E1A62E5FEEB52E28CD0F
:108640008EE00E948B151ECD8EE00E945315B1E086
:108650009B2AAA24AA94BB240FCD8CE00E94531518
:10866000992402CD82E00E94531540909B054194CD
:10867000992493946DCB80E20E945315992444244D
:10868000FF2455245DCB6091A90681E141E10E9460
:108690004C29AECD6091A90682E142E10E944C29AD
:1086A000A1CD6091A90680E145E00E944C2994CDBE
:1086B0006091A9068FE044E00E944C2987CD0E947A
:1086C000021682E20E9453153092700481E20E94E9
:1086D000531580916604882309F47DC082E00E94CE
:1086E0006F1581E00E9427026BCD8BE00E9453152D
:1086F0009924A5CB84E00E946029D5CDEE2009F411
:1087000038CD860107C00F5F1F4F802F8C198E1543
:1087100008F02FCD0E94E000F82EEFE3E81798F361
:108720000E94E000682D0E94D745F301E90FF11D7A
:10873000F0808F2D90E08F7090708D309105B9F0A2
:108740000E9791F09F2D9A21D8018C918B21982B17
:108750009C93D9CFF7EFFF22FFCCE7EFFE228F2DBE
:1087600090E08F709070F5CC87EFF822EBCFF7EFA9
:10877000FF228F2D90E08F709070E2CF82E00E94F8
:108780008B158091C2066091030740911F062091CE
:10879000250609E616E00E94E72B40912506C80150
:1087A000B6010E94E43BE82E1092660435CD8E2D72
:1087B000869509F425CBD6016E2D6150262F281BF6
:1087C0008C91F601E60FF11D90819D93808361509D
:1087D0006217B1F715CB82E00E948B1582CF82E041
:1087E0000E948B158091C2066091030740911F067D
:1087F0002091250609E616E00E945C2C1092660482
:1088000001CDF39481E0F8228DE00E948B15FF20CA
:1088100009F07BC088240E945717C2CA82E00E94D8
:108820008B1559CD6091250689E696E0A6012DE9C4
:1088300035E00E946E29E82E882311F1860106C0DA
:108840000F5F1F4F802F8C198E15D0F40E94E0000F
:10885000F82EBFE3B817A0F30E94E000F8012081D2
:108860006E2D0E94D745F601E90FF11D8081D801D8
:108870008C9320830F5F1F4F802F8C198E1530F340
:108880006091250689E696E0A6012DE935E00E9473
:108890004F2A4091250689E696E0B6010E94E43B06
:1088A000AFCAEE2009F4ACCA860107C00F5F1F4FA4
:1088B000802F8C198E1508F0A3CA0E94E000F82EB4
:1088C0008FE38F1598F30E94E000D8012C916E2D54
:1088D0000E94D745F601E90FF11D80818A219B2D69
:1088E0009223892B8C9380818B212A21822B808358
:1088F000DDCF8DE00E9453158FED95E0B3014091DF
:1089000060040E94E43B882E53CC8DE00E945315F6
:108910008FED95E0B301409160040E94E43B882E06
:108920004091250689E696E0B6010E94E43BE82ED8
:10893000A3E09A2E44246FCF81E00E946029D3C91E
:10894000EF92FF920F931F930E94A614809110073D
:10895000882309F428C184E00E946029FF24F3944D
:1089600007C0113009F472C00E947E2B8823C9F021
:108970000E94A6141091A9061330D9F0143088F380
:108980001430E9F11D3081F781E00E946F30809151
:10899000A9068D3049F3109270040E947E2B882323
:1089A00039F70E944D2B0E94A6141091A90613308E
:1089B00029F70E946629882309F0B2C00E94D82AAC
:1089C000882321F010926204109270040E948C138C
:1089D000882309F092C080911007882329F686E148
:1089E0000E94F712882309F0D3C086E10E940D137C
:1089F000882309F4B9CF80E00E94D61CB5CF0E942D
:108A00006629882309F0A0C080E00E946F30882387
:108A100009F497C08091A906843011F01092700477
:108A200080911007882309F4ABC080916F048130D6
:108A300009F09ACF10926F040E94AB28882309F4A2
:108A400093CF1F910F91FF90EF9008950E94662998
:108A50008823B9F580E00E946F30182F86E10E94CC
:108A6000F712882319F586E10E940D138823D1F4AB
:108A70001123A9F08091A906813011F010927004A1
:108A800080911007882309F07FC00E94AB288823BB
:108A900009F46ACF1F910F91FF90EF9008950E9403
:108AA0006B2BE8CF80E00E94D61CE2CF80E00E94D2
:108AB00044299091B106890F60E040E00E94BF1CFC
:108AC000D2CF0E94021682E20E94531510937004C6
:108AD00081E20E948B1580911F06609125064091CE
:108AE00098052091260600911F06E09096050E94A9
:108AF000461881E00E942702ADCF182F11500E9426
:108B00003717812F0E940E171093AA068091100725
:108B1000882309F060CF8091AA068093B1065BCFCD
:108B20000E940216F092620481E00E94270284E211
:108B30000E9453158091AA060E940E17F0927004AD
:108B40003DCF0E946B2B66CF0E94021682E20E94EC
:108B50005315F092700481E20E94531580911F0614
:108B600060912506409198052091260600911F06E8
:108B7000E09096050E94461881E00E94270244CFAB
:108B800081E00E94602951CF84E00E9460297DCF5E
:108B900080E00E9444299091B106890F60E040E096
:108BA0000E94BF1C22CF81E00E946029D7CE991B72
:108BB00079E004C0991F961708F0961B881F7A95D4
:108BC000C9F780950895AA1BBB1B51E107C0AA1FD6
:108BD000BB1FA617B70710F0A61BB70B881F991F5E
:108BE0005A95A9F780959095BC01CD01089597FB02
:108BF000092E07260AD077FD04D0E5DF06D0002035
:108C00001AF4709561957F4F0895F6F790958195C8
:108C10009F4F0895A1E21A2EAA1BBB1BFD010DC098
:108C2000AA1FBB1FEE1FFF1FA217B307E407F5071C
:108C300020F0A21BB30BE40BF50B661F771F881FF8
:108C4000991F1A9469F760957095809590959B018E
:0C8C5000AC01BD01CF010895F894FFCFE6
:108C5C000100010001000100010001000100010000
:108C6C000100010001000100010001C00080004072
:108C7C00007F206430480F04050607111210130EF4
:108C8C0004050607111210130409050A06070B1137
:108C9C000C120D101325212326272422201D1E1B08
:108CAC00191F1C1A1012180F110C130E0B140D0A8D
:108CBC0015160917040508030601070002032019FD
:108CCC001A180C0B0A090420191A180C0B0A092281
:108CDC0021252320191A18241B1C0F0E0D04030A1E
:108CEC000C0B0908010200201B191C1A180F0C0E82
:108CFC000B0D0A0926271D1E1F1012111314151611
:108D0C00170506076E306E783078000100070E09E3
:108D1C001C1B1215383F363124232A2D70777E798F
:108D2C006C6B6265484F464154535A5DE0E7EEE97F
:108D3C00FCFBF2F5D8DFD6D1C4C3CACD90979E996F
:108D4C008C8B8285A8AFA6A1B4B3BABDC7C0C9CE5F
:108D5C00DBDCD5D2FFF8F1F6E3E4EDEAB7B0B9BE4F
:108D6C00ABACA5A28F88818693949D9A2720292E3F
:108D7C003B3C35321F18111603040D0A5750595E2F
:108D8C004B4C45426F68616673747D7A898E87801F
:108D9C0095929B9CB1B6BFB8ADAAA3A4F9FEF7F00F
:108DAC00E5E2EBECC1C6CFC8DDDAD3D4696E6760FF
:108DBC0075727B7C51565F584D4A4344191E1710EF
:108DCC0005020B0C21262F283D3A33344E494047DF
:108DDC0052555C5B7671787F6A6D64633E393037CF
:108DEC0022252C2B0601080F1A1D1413AEA9A0A7BF
:108DFC00B2B5BCBB9691989F8A8D8483DED9D0D7AF
:108E0C00C2C5CCCBE6E1E8EFFAFDF4F30409050AA0
:108E1C0006070B110C120D101300010001000100CC
:108E2C00010001000100010001000100010001002E
:108E3C00010001C000800040000606011718191A35
:108E4C001B1C1D1E1F202122233F3F3F0B0C0D0E10
:108E5C000F10111213141516173F3F3F232425260C
:108E6C002728292A2B2C2D2E2F3F3F3F1718191A54
:0E8E7C001B1C1D1E1F202122233F3F3F1500FF
:00000001FF
